:020000040800F2
:10500000F81B0020D5500008A18C000891830008EF
:105010000000000000000000000000000000000090
:10502000000000000000000000000000E59A0008F9
:10503000000000000000000061940008219C0008AE
:10504000E7500008E7500008E7500008E750000864
:10505000E7500008895D0008E7500008E7500008A5
:1050600000000000E7500008B15C0008E7500008AD
:10507000E75000089188000800000000E750000891
:1050800000000000E75000080000000000000000E1
:10509000E750000800000000E7500008E750000853
:1050A000E7500008E7500008E7500008B9A60008DC
:1050B000E7500008E7500008000000000000000072
:1050C0000348854600F040FD004800472DBA00081F
:1050D000F81B00200448804704480047FEE7FEE72D
:1050E000FEE7FEE7FEE7FEE7BD9C0008C1500008B2
:1050F00030B50B46014600202022012409E00D4670
:10510000D5409D4205D31D469540491B25469540F7
:1051100040191546521E002DF1DC30BDF0B51FB40C
:105120000646002082B005464024019100901BE015
:10513000019922460F46304600F0F0FB049A059B89
:10514000801A994110D310461946224600F0D6FB2A
:10515000361A8F410197224601200021009F00F05E
:10516000CDFB38184D4100902046641E0028DFDC3E
:10517000019B00982946324607B0F0BD03460B4319
:105180009B0703D009E008C9121F08C0042AFAD2FD
:1051900003E00B780370401C491C521EF9D2704783
:1051A000D2B201E00270401C491EFBD270470022BF
:1051B000F6E710B513460A4604461946FFF7F0FF16
:1051C000204610BD30B504460020034600E05B1CBD
:1051D000934203D2E05CCD5C401BF8D030BDF8B503
:1051E00002464A40D40F42004B0052085B089A42E4
:1051F00002D20246084611464A0023D0C30D4A0097
:10520000DDB2120EAD1A202D35DA49020126490A07
:10521000F6058A19002C00D0524220214F1B11465E
:10522000B9402A411018C20D9A4221D0002C17D043
:10523000012D08DCDA05801AD20F8019D207DBB203
:1052400000F098FBF8BDDA05801A012340001B0628
:10525000C01880185A428018CA0F1043490007E04E
:105260004908C2071143DA05801A801940088018DE
:1052700000F078FBF8BD61000122511A001BF7E72E
:105280000122D2075140AAE70122D2075040A6E7E7
:10529000024670B54A40D30FDB0740002DD04A00CC
:1052A0002AD0010E140E000212020919400A520AF5
:1052B0008418E50104465443000A120A2E045043A0
:1052C000A4194219200CC543AA18120C0125AD03DC
:1052D000521C521912047F39240400D0521C10436E
:1052E00001D44000491EC2B20C06C0092018401C5F
:1052F0004008802A02D003E0002070BD4008400032
:10530000002900DA0020184370BD70B502464A40FB
:10531000D50F40004A00ED0740085208002814D07D
:10532000002A12D0C40DD30D41020120C005520243
:10533000490A520AE41A091812187D34914201D31D
:10534000641C00E04900002C01DA002070BD00233D
:10535000914201D3891A0343400849000028F7D13C
:1053600000290AD0914202D10121C90705E09142EA
:1053700001D2012101E00121C943E005C018401913
:1053800000F0F0FA70BD420005D04200120E524209
:105390008A4201DB00207047C905081870470000E9
:1053A000F0B507460846584087B0C00F0490480043
:1053B0000E46590040084908BC1A884105D23846B3
:1053C00031461E4617460B46024658004008104319
:1053D0004CD0300D039040055900400D490D05900B
:1053E000401A0290402872DA18030121000B0905C7
:1053F0000843019004980092002805D00199524278
:105400000020884100920190029840210A1A0199D7
:10541000009800F073FA05460C466B4607CB00F087
:105420008EFAC0197141039A0E0D0023D71756400A
:105430001A467A40164344D0049A002A2DD0029A84
:10544000012A039A15DC1205C01A9141012636057E
:10545000001C7141D20F059ED20700930192029663
:105460002A46234600F0CCFA07B0F0BD3846314654
:10547000FAE71605224A0F46B218C01AB7410121B1
:105480000905001C4F4100187F4111461818794149
:10549000E20F10436D19644113E0E2076D081543F4
:1054A0006408C2071443039A01261205C01A9141E9
:1054B0003605001C7141CE07400830434908C0182A
:1054C00051412A46234600F08EFACDE7FFE70498C3
:1054D00001224000C117121A00238B410498314663
:1054E000C417381AA141EEE730B40124E407634041
:1054F00030BC55E730B40124E407614030BC4FE7CD
:105500000000E0FFF0B51FB488B00B9909980024A3
:1055100048400999C00F490049080991C0070B99F3
:105520000090490049080B9109990898A64608433C
:105530001CD00B990A98084318D009980124400000
:10554000420D4800410D099824050003000B20433B
:1055500009900B980003000B20430B9050181C4936
:105560004018002201901446104605E00020014634
:105570000DB0F0BD032801DA034600E003239C468A
:10558000C11A0AAE0AE05F0008ADED5B4F00F75BA1
:105590007D430027AA187C41491C5B1E6145F2DD52
:1055A000410004AB5A522104120C0A43240C401C43
:1055B0000828DFDB01980290009970460191009065
:1055C000059B049A0799069800F01AFAD0E70000A4
:1055D0000DFCFFFFF0B50C465C4085B0E40FE4071E
:1055E00003944C000026640859009446490802467A
:1055F0000296224321D062460A431ED06200570D14
:105600004A000E032303550D012402462C492405AC
:10561000781B1B0B360B4018234326436146009032
:105620001C46501AB44103D30098401C009002E07D
:10563000921800985B41002803DA0020014605B06B
:10564000F0BD0020012109050746864611E06446A9
:105650001D46141BB54106D36546521BB341744623
:1056600007430C43A646CD07400849082843921833
:105670005B4105460D43EAD11046184313D06046FE
:10568000194650407140084306D06046101AB34195
:1056900006D20122002306E000220123DB0702E0FC
:1056A0000122D2435310009874460105381C614111
:1056B000029C039D0019694100F095F9BFE70000C5
:1056C000FD03000070B54B005B0803430BD04B009B
:1056D0005C0D002633466542B341D417AD1AA34191
:1056E00002DB0020014670BD12053018514170BD2B
:1056F000C217C10F504010B54018CA0796230021A9
:1057000000F038F910BD10B500229623114600F0C4
:1057100031F910BD0EB5C217C10F5040CA0740186D
:105720000021054B0293019200910A460B4600F0BE
:1057300067F903B000BD0000330400000EB5054951
:105740000291002100910A460B46019100F058F9A0
:1057500003B000BD33040000C20F4100400201232A
:10576000400ADB05D207090EC0187F2901DA0020A4
:105770007047962903DC9623591AC84001E09639F0
:105780008840002AF4D04042704741004002012284
:10579000400AD205090E80187F2901DA00207047DF
:1057A000962903DC9622511AC840704796398840E2
:1057B0007047000070B5CD0F4A0009030123090BA3
:1057C0001B0519430B4BED070024520D9A4201DAD9
:1057D000002070BD074B34339A4203DC9A1A00F064
:1057E0009DF802E00449511888402C43F1D0404212
:1057F00070BD0000FF030000CDFBFFFF4A0009035E
:105800000123090B1B051943094B10B5520D9A4290
:1058100001DA002010BD064B34339A4203DC9A1A99
:1058200000F07CF810BD03495118884010BD0000FD
:10583000FF030000CDFBFFFFC20FD207400040086E
:105840000BD0C10D0723DB01C91840020905400A2E
:105850001143C208400711437047002001467047BA
:1058600010B5002904DB0124E40740428C412146A5
:10587000002B04DB1C460123DB075242A3418B4271
:1058800000D1824210BD000010B5002904DB0124C4
:10589000E40740428C412146002B04DB1C460123D7
:1058A000DB075242A341994200D1904210BD000053
:1058B000CB0FDB07490010B5490802460A4307D061
:1058C0000A0D07240903E401090B121B002A01DC5D
:1058D000002010BDC900440F0C43C100E018D205E0
:1058E000801800F03FF810BD0122D207002800DB2D
:1058F000101A002900DB511A8142704710B5202A86
:1059000004DB0146203A9140002010BD9140202345
:105910009C1A0346E3401943904010BD10B5202A5D
:1059200004DB0846203AD040002110BD0B46D3408E
:10593000D0402024A21A91400843194610BD10B54A
:10594000202A06DBCB170846203A1041C1170B432B
:1059500006E00B461341D0402024A21A9140084390
:10596000194610BD002904DA401C490001D1400845
:105970004000704770B40024050C05D110240004C9
:1059800002D1002921D01124050E01D100020834D2
:10599000050F01D10001241D850F01D18000A41C39
:1059A000002801DB4000641C002908D020252E1BA4
:1059B0000D46F540A14000D00121294308430106CE
:1059C0001B1B000ADB1D02D5002070BC7047DB05E5
:1059D000181880180029F8DA401C4900F5D170BC6D
:1059E00040084000704710B5002B08DA0024401C26
:1059F000614192185B411A4301D14008400010BD3B
:105A0000F0B51FB482B005460C0003D0084604F080
:105A100007FF02E004F004FF203002460090214618
:105A20002846FFF76BFF049B059A04460F46184370
:105A30001143084314D0184610431BD0009840214E
:105A40000A1A18460599FFF769FF05460E46009A9F
:105A500005990498FFF752FF084305D0012004E0A0
:105A60002046394607B0F0BD0020C11705430E435C
:105A70002C43374300990E986305401A7905E40AD0
:105A800000220C43FD0A0A3002D500200146E9E756
:105A90000105101969410C9C0D9D00196941FFF722
:105AA000A2FFDFE7FEB500231A461B1A8A4103DB7B
:105AB0000020014603B0F0BD4A000D0301212D0B6B
:105AC0000905520D0D43D10702D100186D41521E38
:105AD0005110FF31FF310131002704463E46384660
:105AE000009701910246012100200905FFF716FFEA
:105AF000C3197141F818324684468E464A416146C0
:105B00002846611A904104D36046241A954176468E
:105B10001F46241900986D41401C00903428E1DD97
:105B2000F91930467041091BA84103D20022D24323
:105B3000134601E00022134601980105381C71410B
:105B4000FFF751FFB6E70000064C0125064E05E0C1
:105B5000E36807CC2B430C3C98471034B442F7D38E
:105B6000FFF7B2FA10C9000830C9000870B58C18E8
:105B70000578401C6B075B0F01D10378401C2A118C
:105B800006D10278401C03E006780E70401C491CC8
:105B90005B1EF9D12B0705D40023521E0DD40B70C8
:105BA000491CFAE70378401CCB1A921C03E01D78CD
:105BB0000D70491C5B1C521EF9D5A142D8D30020A0
:105BC00070BD000038B50446064805490068FFF777
:105BD0008FFA604300E0401E00900028FBD138BDE2
:105BE00040420F0084010020F8B504460068816837
:105BF0008907890F012902D10168C90722D181686B
:105C0000114A10261140012500290ED1816829432F
:105C100081600120FFF7D6FF01F028F807460CE06D
:105C200001F024F8C01B0A2807D9606D3043606575
:105C3000A06D2843A0650120F8BD20680068C0431E
:105C4000C007EDD10020F8BD170000801FB50B483C
:105C500000900B4801900B4802900B480390694656
:105C60000A4805F0D3F90A4A08481146083905F0F0
:105C7000BBF800F06FFA002004B010BD1DC700088B
:105C8000F9C6000859C7000857C70008900100204E
:105C90001000002010B500231A4603E0845CE318CE
:105CA0009BB2521C8A42F9D3D84380B210BD000087
:105CB00010B5034800F096FD024800F093FD10BDBA
:105CC000981700205017002030B5446C1C252C403C
:105CD0000125A540046C6560046863608368102B2F
:105CE000036803D099600068C26030BD9A600068A4
:105CF000C16030BD1449012048720A4602205E325C
:105D0000507203203C3A507204200E3A50720F48F1
:105D10000D4B0078087022310870203108770C494B
:105D20005A1C087858714978997123331871597140
:105D3000203318775977107551751A461E32107531
:105D40005175107651767047E81100203E01002011
:105D50006001002010B503F09BFE202003F056FFE9
:105D6000012005F0BDFB002003F050FF044805F0C2
:105D70005BFA044805F00AFD002005F03FFD10BD68
:105D80000001002083800000F8B503F04DFF0520DE
:105D90000121000700F056FF0025144C002800D018
:105DA0006560134E0221304600F04CFF002815D1EB
:105DB000012020700F48808F00280ED00127BF02DD
:105DC00000223946304600F04AFF0A2004F07CFFEA
:105DD00001223946304600F042FF6560012000F0A4
:105DE00069FE022000F066FEF8BD00007001002090
:105DF00000040050E80D00207047000010B508496D
:105E000000224A6107494B684C1523434B604B689D
:105E1000082423434B60C009C001026010BD00008C
:105E2000E0170020002002407FB500250C46064602
:105E3000039500F00FFEE009029003A9019600957A
:105E4000684600F09FFD002804D000F0D7FD002038
:105E500004B070BD00F0D2FD0120F9E710B50023B9
:105E600002E0C45CCC545B1C9342FAD310BD00002A
:105E700010B5214A00219069C305204804D5416925
:105E8000022319434161911593699B0505D5436927
:105E90000124234343616302194393695B0505D5DC
:105EA0004369082423434361E301194393691B05B4
:105EB00005D543690424234343616302194393696D
:105EC0009B0405D5436910242343436163021943AE
:105ED00093699B0304D5446920231C4344611943FF
:105EE0009369DB0305D54369402423434361A00242
:105EF0000143916110BD000000200240E017002026
:105F000070B5054600F0B2FE0646184C0AE0681C63
:105F100008D0002D04D000F0A9FE801BA84201D9B2
:105F2000032070BDA069C007F1D1A069800701D529
:105F30000220A061A069C00511D4A06980050ED41B
:105F4000A06940050BD4A069000508D4A0698004AD
:105F500005D4A069800302D4A069C00303D5FFF76C
:105F600087FF012070BD002070BD000000200240AE
:105F7000F8B51746002605460C4600F06BFD09E013
:105F800029460220226800F047FD002804D1241D84
:105F90002D1D361DBE42F3D300F030FDBE4201D2AE
:105FA0000020F8BD0120F8BD10B5084902460020C8
:105FB000054B497905E044001C5B944203D0401C2A
:105FC000C0B28842F7D310BD8C13002070000020AF
:105FD00010B500F03CFE10BD10B5094801F05CF8AA
:105FE00080B2FFF7ABFB074A074BFFF78BFA0022A3
:105FF000064BFFF7EFFAFFF701FC80B210BD00007F
:1060000004160020F853E3A59B843E4000408F40D7
:1060100070B50024204603F0BBF947494748A20069
:10602000641CE4B28150142CF9D3464944480A79DF
:1060300002754979417544490A7802764978417672
:106040003F490520133148720A2005F08FFB7D205F
:10605000400105F0A5FB3A49002213310C2005F060
:106060006FFC00210C2005F07DFC384801F014F88D
:10607000344C0125203CE084AD0309E0334801F0B5
:106080000BF880B2E084A18EFF392D39884206DBFF
:10609000A18E80B28842F1D349198842EED80220FD
:1060A00005F0B4FB002003F073F9294D00210F2007
:1060B00005F0DCFA2842E063F8D0E06B411C38D0F0
:1060C000400435D58122D20100210F2005F00DFCBE
:1060D0000021102005F0CAFA41061948490E002295
:1060E000C73005F0F9FA164DC735687A05281FD173
:1060F00002221549681DFFF765F8002818D11148DC
:10610000AE7C66710422691C3430FFF737F82946EB
:106110001331084672000D466930FFF72FF8607999
:106120002946420005484838FFF728F80320207028
:1061300070BD04F0E9FB0000FFFF0100EC1300203C
:106140004912002090000020600100200416002069
:1061500000D0272410B5144C1448224610321146A2
:10616000083904F041FE0022114BE168A068FFF7F6
:1061700031FA104A104B05F061FD00220F4BFFF77A
:10618000B9F900220E4BFFF7BDF9FFF791FB206034
:1061900000221346E168A068FFF762FB01D0206887
:1061A00010BD0020206010BD0000002090010020E4
:1061B00000AA8F406C45D9CC955BC83F0000F03FEA
:1061C00040A5E54010B5084800F096FA0A210648B7
:1061D00000F032FA044800F01DF9800503D50248AA
:1061E00000F01AF980B210BDA8150020F8B52F4DA7
:1061F00000220121284600F032FDFFF7E3FFFFF700
:1062000082FA2B4E3146FFF780F82A4C0122A0601B
:106210001146284600F023FD2749A0680025884242
:106220003EDB2078254F002815D02570FFF7CAFFE8
:10623000FFF769FA3146FFF768F8A060FFF7FCFA4C
:1062400000223B46FFF750F900221D4BFFF75AF999
:10625000FFF72EFB6060A068FFF7EEFA00223B46D6
:10626000FFF742F9174A184BFFF74CF906460F465D
:106270006068FFF7E1FA134A144B5242FFF742F904
:1062800032463B46FFF78CF8FFF712FB104960607F
:10629000884201DD616004E0FF21C905C84200D3E6
:1062A00065606068FFF771FAC0B2F8BD0004005085
:1062B00000401B44480000200000604000000C40EB
:1062C00000E064403333333333B33040CCCCEC3F65
:1062D0000000C842F8B5054604464035287C002633
:1062E000012808D001202874206881688907890F57
:1062F00001290ED101E00220F8BD0168C90708D0CC
:10630000606D202108436065012600202874304616
:10631000F8BD616DFF220132914302221143616594
:10632000C1688907890F0091C16889088900C16027
:106330002068816892071143816000F097FC07464E
:106340000EE000F093FCC01B0A2809D9606D022101
:106350008843102108436065002028740120F8BD9F
:10636000206880680028ECDB2068C168009A11432F
:10637000C160606D80088000401C6065C5E700005A
:10638000F8B506460D464036317C01290DD0012175
:10639000317401688A68520709D5416D2022114382
:1063A0004165002030740120F8BD0220F8BD174B74
:1063B0006A68D80547109A42154C8A6A2B6812D031
:1063C0005B035B0B1A438A622968490305D5A16800
:1063D0000143A1600A20FFF7F5FB2868800312D56E
:1063E000A06838430EE05B035B0B9A438A6229681E
:1063F000490302D5A1688143A1602868800302D5C2
:10640000A068B843A06000203074F8BD01100000FF
:1064100000270140406D70470068006C7047000025
:1064200070B5040006D0606D264600254036002871
:1064300002D006E0012070BDA5653574204600F04D
:10644000D3F8606DC00603D421688868400705D57D
:10645000606D1021084360653574EBE7606DFF22C5
:106460000132904302221043606588688207920FD0
:106470005B48012A02D10A68D2072BD10323626844
:106480009B079A4205D05B429A4202D05B009A4237
:1064900009D10A69920092080A6121680A69636851
:1064A0001A430A610CE00A69920092080A61816845
:1064B0000F22920491438160816862681143816078
:1064C0002168CA6818239A43CA602168CA68A36809
:1064D0001A43CA6081680122520691438160816833
:1064E000A28E52061143816020688168C90004D4DD
:1064F000816801221207114381602068C168394A0E
:106500001140C1602069E168022825D000200143C4
:10651000204620300278037B52035B001A4311436C
:10652000226B1143A26992031143E269D203114322
:106530002268D3681943D160616A0A46FF3AC23AB9
:1065400005D0A26A11432268D3681943D16042780A
:106550000121012A02D00BE00420D8E700780028AE
:1065600023D0606D202210436065A06D0843A065B4
:10657000E06B012820681FD00169C90703D00169B9
:1065800049084900016120684169C908C9004161A1
:1065900020684169A26B11434161A565606D800867
:1065A0008000401C6065002070BD2068C268012327
:1065B0001B041A43C260DBE70269FF239B009A4376
:1065C000026120680269236CA66C1A43636C334332
:1065D0001A430261206802690A430261D3E700009E
:1065E000002701401902FEFF10B586B004461421B1
:1065F0006846FEF7DCFD0E492068884216D10D483A
:10660000416B421511434163C16A01221143C162CA
:10661000C06A694610400590022000900320019056
:10662000002002900520000700F050FA06B010BDCF
:106630000024014000100240F8B504464069254698
:1066400040350E4608280BD02068C068C00709D026
:10665000606D202108436065002028740120F8BD8A
:10666000082700E00C2700F001FB009011E0701CEF
:106670000FD0002E05D000F0F9FA0099401AB04270
:1066800007D9606D04210843606500202874032049
:10669000F8BD206800683842E9D0606D01214902E8
:1066A000084360652068C16809058A0F0C21002A2B
:1066B0001BD12022125D002A17D10268120714D5BF
:1066C000826853070122002B08DB43688B43436039
:1066D000606D130298431043606506E0606D2023EF
:1066E00018436065A06D1043A065A069002801D122
:1066F000206801600020F8BD70B5044621680020C4
:106700008968490721D425464035297C01291CD0B8
:1067100001212974E169012904D02046FFF764FAB8
:10672000002811D1616D0A4A1140FF220132114344
:1067300061650021A165297422681C21116021680E
:106740008A6804231A438A6070BD022070BD00006D
:10675000FEF1FFFF30B5014620314A790023022ABD
:1067600004D00422C2630B71012030BD026814689A
:106770000E25AC4314600268146864086400146059
:10678000446C1C22144001221546006CA540456053
:106790004A7118460B7130BD70B500240146203196
:1067A0004A79022A03D00421C163012418E0026857
:1067B00013680E25AB431360026813685B085B0027
:1067C0001360436C1C221340012215469D40036C4C
:1067D0005D604A7100220A71816B002900D08847F0
:1067E000204670BDF0B4016C0D6801680C68466C01
:1067F0001C2304221E401746B7402F420ED06707C5
:106800000CD50C68A40602D40C6894430C60416C4F
:1068100019408A40016C4A60016B1AE00227B740B8
:1068200002462F402032002F17D0A70715D50C683D
:10683000A40605D40C680A25AC430C6001215171F3
:10684000446C02211C40036CA1405960002111716D
:10685000C16A002918D0F0BC08470827B7402F426A
:1068600012D0240710D50C680E25AC430C60446C84
:1068700001211C400B46A340046C6360C16351714D
:1068800000211171416BE4E7F0BC704770B5040062
:106890003CD01F48256814212818FEF729FC8000E9
:1068A00060641C4820640221204620300246417169
:1068B00029681948E3680140A0686669184323699C
:1068C00033431843A3691843E3691843236A184301
:1068D000084328600121A0688903884210D00D4830
:1068E0008030836A656C1C210D400F26AE40B34397
:1068F0008362656C63680D40816AAB400B438362C1
:106900000020E06301215171107170BD012070BD44
:10691000F8FFFDBF000002400F80FFFFF8B50446FE
:106920008C46203001790025012909D00126067105
:1069300041790027012905D0077102252846F8BDB5
:106940000220F8BD02214171E7632068016849080F
:106950004900016061462046FFF7B6F9206B002828
:106960002068016801D00E2205E0042291430160F5
:10697000206801680A2211430160206801683143E0
:106980000160DBE7F8B51A4E0546307C0F4601285A
:1069900007D0012030741748FFF7B2FA010002D087
:1069A00021E00220F8BD0020C04338606C6814E08C
:1069B0002046FFF723FA0F48FFF7A2FA01460E48D8
:1069C000426808239A434260426843159A434260F2
:1069D000002901D03C6006E08034A8686A68C001E4
:1069E0008018A042E4D8002030740846F8BD0000AA
:1069F000E017002050C30000002002400548416815
:106A0000022211434160416801221143416000208C
:106A10007047000000200240F8B50C4C1646207C60
:106A20000F46012808D0012020740948FFF768FAB2
:106A30000025002802D006E00220F8BD65613E6016
:106A40000348FFF75DFA2574F8BD0000E017002049
:106A500050C3000011484168C9070BD0EFF3108103
:106A600072B60F4AC2600F4AC26081F31088416853
:106A7000C9070ED1416889070DD5EFF3108172B6B1
:106A8000094A0261094A026181F31088406880075F
:106A900001D501207047002070470000002002400F
:106AA000EFCDAB8905040302BFAE9D8C1615141300
:106AB0007047000010B504494A69024202D048619B
:106AC000FFF7F6FF10BD000000040140FCB50023F5
:106AD0000124A2E027462A469F403A406FD04D68E5
:106AE000012D05D0022D03D0112D01D0122D16D16C
:106AF00085680326AC465D00AE46AE406546B543AC
:106B0000AC46CE687546AE4065462E438660466804
:106B10000D79BE43ED06ED0F9D4035434560C668D7
:106B20005F000325BD40AE46AE4335468E68BE408D
:106B30002E43C6604E68022E01D0122E14D1DE08FC
:106B4000B60036180196366A5D07B446EE0E0F257C
:106B5000B54000966646AE43B4460D69009EB5400A
:106B600066462E43019D2E6206687546AE430D793A
:106B7000AD07AD0FBD40354305604D68ED004BD509
:106B8000294D6E6B26436E639E08284DB60075191D
:106B9000AC46AD689E07360F0F27B740BD430527AB
:106BA0003F07B84201D1002715E0214FB84201D17B
:106BB000012710E01F4FB84202D102270BE02BE063
:106BC0001D4FB84201D1032705E01C4FB84201D147
:106BD000052700E00627B7402F436546AF60184DF4
:106BE0002E684F689643FF0300D516432E606E68EB
:106BF0004F689643BF0300D516436E60AE684F687A
:106C00009643FF0200D51643AE60EE684F68964388
:106C1000BF0200D51643EE605B1C0A681546DA40D9
:106C200000D057E7FCBD000000100240000001400A
:106C30000004005000080050000C0050001C0050E0
:106C4000000401400069084000D0012070474269FB
:106C500013460B401B0491430B4383617047002A8A
:106C600001D08161704781627047000001488068EF
:106C70007047000078010020024881680278891876
:106C8000816070477801002010B508480024016831
:106C9000402211430160204600F00AF8002801D08C
:106CA000012401E000F042FA204610BD002002401D
:106CB00070B504460D4D7D202978C000FEF718FA06
:106CC00001460B480068FEF713FA00F02BFF00287E
:106CD00009D1042C07D200222146401E00F04EFAB2
:106CE00000206C6070BD012070BD000078010020A4
:106CF0008401002070477047F8B502F095FF604CA2
:106D00000120E070208AFEF7FEFC01467F20C005CE
:106D1000FEF7FBFA5B4D06462968FEF760FA28602D
:106D20000120A16AC005814201DA084603E030462D
:106D3000FEF7AAFAA062FF21C9050025C84200D3C8
:106D4000A562607800280BD102214F48FFF77AFF37
:106D500002004E494E4817D00022FFF780FFE5623F
:106D600002214948FFF76EFF4A4E002855D0E562E0
:106D7000B08AFEF7C8FC434F3968FEF7B5FD5FD215
:106D80004549012008705DE00122D1034048FFF72A
:106D900066FF208AFEF7B7FC01467F20C005FEF79C
:106DA000B4FAE16AFEF71BFA3C49E0628842D7DD9B
:106DB00038480127F926403000900A213046FEF776
:106DC00097F9002903D131493148FFF701F9022130
:106DD0002D48FFF737FF002801D0002701E0002FE2
:106DE00012D102212848FFF72DFF00280CD104F012
:106DF000EDFE00990120888005F044FC642003F03A
:106E000063FF28492648C8600A2003F05DFF30462A
:106E1000761EF6B20028D0D1A2E7208AFEF773FCD6
:106E200001467F20C005FEF770FAE16AFEF7D7F948
:106E30001D49E06288429BDB1A491948C86097E700
:106E400015480570708F401EFEF752FC3968FEF73A
:106E50004BFD06D82079002803D014490120087082
:106E600001E012480570708FFEF74DFC3968FEF79F
:106E70003BFD04D22079002801D004F06BFEF8BD60
:106E80003C0100207401002000040050008000003C
:106E900000000050E80D0020760000200000404077
:106EA0000400FA0500ED00E00000A040830000208F
:106EB000704770B5040010D0022025462035A87315
:106EC000204601F0EDFCA87B032805D0204600F009
:106ED000B9F80020A873687370BD012070BD7047B9
:106EE000704710B5044600680168C943C90708D156
:106EF0008168C943C90704D1012141602046FFF7D9
:106F0000FBFE20680168C943890708D48168C9432A
:106F1000890704D4022141602046FFF7EBFE206878
:106F20000168C943490708D48168C943490704D4A3
:106F300004214160204600F0F7F820680168C94349
:106F4000090708D48168C943090704D408214160AE
:106F50002046FFF7ADFF20680168C943C90608D481
:106F60008168C943C90604D4102141602046FFF757
:106F7000C2FE20680168C943890608D48168C943F4
:106F8000890604D4202141602046FFF7A9FF20682C
:106F90000168C943490608D48168C943490604D435
:106FA000402141602046FFF79AFF10BDF8B504006C
:106FB00005D025462035A87B002802D006E0012018
:106FC000F8BD00206873204600F04EF80220A87338
:106FD0002068C26884466368012B01D10620824381
:106FE00016486169814202D0072040038243002B8A
:106FF00001D1D82082431248A66802401846304387
:10700000676A266A3E433043A66A30431043002B2A
:1070100002D0012B04D005E02369E2691A4300E0A5
:10702000E2681043054A914202D0A2691143084325
:107030006146C8600120A8730020F8BDFFFF000072
:10704000F8F119FF10B500680549884207D10548D5
:10705000816B4900490881630D2000F073F810BD71
:10706000007C00400010024010B5006808498842CA
:107070000CD10848816BC2041143816300220121B5
:107080000D2000F07BF80D2000F06CF810BD000022
:10709000007C0040001002400068C069704700009A
:1070A000F8B504460220254620351746A8731D482A
:1070B0000268C3041A4302602068C2689B121A4324
:1070C000C2602068026901263243026122681020F2
:1070D0005060206881611021204601F051FC032896
:1070E0001FD0216808204860206847610821204699
:1070F00001F046FC032814D0204601F0D1FBA87B08
:1071000003280ED0206881683143816020680169BE
:107110003143016120680169042211430161AE73AA
:107120000020F8BD00040140704700000448416B96
:10713000012211434163816B020411438163704753
:1071400000100240002809DBC106C90E012088405A
:1071500003490860BFF34F8FBFF36F8F7047000084
:1071600080E100E0002805DBC106C90E012088404F
:10717000014908607047000000E100E010B503F02D
:10718000A1FB10BD02494A6882434A607047000073
:107190000070004002480168821511430160704789
:1071A0000070004002494A6802434A60704700008C
:1071B0000070004005480168022211430160044844
:1071C000016904221143016130BF70470070004023
:1071D00000ED00E0F0B5154A1368154D54152D6A01
:1071E0002340ED07ED0F002B04D0002D02D01668D0
:1071F000A64316601668B608B600064316600D482A
:10720000076904263743076101290DD040BF20BF1D
:1072100020BF0169B1430161002B04D0002D02D0D1
:10722000106820431060F0BD30BFF2E700700040EE
:107230000000014000ED00E0F8B5044600780027AA
:10724000534D800671D5524E403EB06BC00004D401
:10725000B06BA9050843B06301274E480168C90512
:1072600011D40168821511430160FFF7FFFC009003
:1072700005E0FFF7FBFC0099401A642837D8454821
:107280000068C005F5D532680321090560680A4029
:107290000140914208D08103890F032904D131684C
:1072A000890301D50120F8BD2A69032109040A4098
:1072B00022D0084090421FD0207880061CD5286933
:1072C0002A6988430121C9040A432A612A698A4339
:1072D0002A612861C0050FD5FFF7C8FC009008E0BF
:1072E000FFF7C4FC0099411A2B48814201D90320C1
:1072F000F8BD28698005F3D561688803800F0328ED
:1073000005D132680005824301400A433260286992
:10731000032261681204114008432861002F04D041
:10732000B16B012000078143B1632078C00705D00D
:10733000E868A168800880000843E860207880073A
:1073400005D5E8680C218843E1680843E8602078A7
:10735000400706D5E868032189028843216908436C
:10736000E8602078000706D5E86803210903884310
:1073700061690843E8602078000606D5E8680321C3
:1073800089048843A1690843E8600020F8BD000033
:10739000401002400070004088130000F8B50E460F
:1073A000050038D05E480068C007C00FB04214D254
:1073B0005B4C20684008400030432060FFF756FCDB
:1073C000074605E0FFF752FCC11B564881427AD8B8
:1073D0002068C007C00FB042F4D12878524C800713
:1073E00005D5E068F0218843A9680843E060287863
:1073F000C00752D06868022806D0032807D0216849
:1074000001280AD0890504E02168890301E0216888
:107410008901002903DB0120F8BD4907F9E7E1688C
:10742000890889000143E160FFF720FC074668688E
:1074300002280AD0032814D001281ED029E0FFF723
:1074400015FCC11B374881423DD8E0680007800F1A
:107450000228F4D121E0FFF709FCC11B3148814229
:1074600031D8E0680007800F0328F4D115E0FFF75A
:10747000FDFBC11B2B48814225D8E0680007800F27
:107480000128F4D109E0FFF7F1FBC11B2548814237
:1074900019D8E0680007800FF5D121480168C907B5
:1074A000C90FB14217D90168490849003143016049
:1074B000FFF7DCFB074608E005E0FFF7D7FBC11B41
:1074C0001848814201D90320F8BD15480068C0075B
:1074D000C00FB042F1D12878400706D5E0680721F7
:1074E00009028843E9680843E0602878000707D567
:1074F000E0680721C90288432969C9000843E060A0
:1075000000F03AF8E168094A0906090F515CC840E1
:107510000749086007480068FFF7CAFBF8BD00008C
:107520000020024088130000001002405EC80008DE
:10753000840100207C010020044805490068C968D6
:10754000044A4905490F515CC84070478401002036
:107550000010024077C80008044805490068C9685F
:10756000044A8904490F515CC840704784010020D7
:107570000010024077C8000870B51A4AD3681A494B
:107580000C2018408D0004280CD04E00082810D084
:107590000C2810D050680004410F0120C003491C82
:1075A000884070BD1068C00601D5084670BD2846E9
:1075B00070BD304670BD98020C4C000F205C1B0261
:1075C0009C0FD368641CDB0301D5314603E01268CD
:1075D000D20600D4294603F03AF922460023FDF7EB
:1075E0009DFD70BD0010024000093D006EC80008FE
:1075F000FEB505007ED0FE4CE7680C20E66807402B
:107600000120000406402878C00747D0082F05D085
:107610000C2F0AD101200004864206D12068800385
:107620003CD568680028E5D038E00120696800048E
:10763000814203D121680143216011E00523012229
:107640001B0492049942216802D111432160F1E7A1
:1076500081432160216801400091206890432060AF
:10766000686800280DD0FFF701FB009005E0FFF7E8
:10767000FDFA0099401A64287BD820688003F6D56B
:107680000CE0FFF7F3FA009005E0FFF7EFFA00993E
:10769000401A6428F0D820688003F6D42878800740
:1076A00056D50923E868042F0DD00C2F01D1002EE8
:1076B00009D000283CD02168994301432160FFF79D
:1076C000D5FA064628E02168490701D5002891D05F
:1076D00061681F22120291432A69120211436160FC
:1076E0002168994301432160FFF746FFE1680906DD
:1076F0000A0F00E08BE1BF49895CC840BE490860C1
:10770000BE480068FFF7D4FA002873D120E0FFF7E5
:10771000ADFA801B0228AFD820684007F7D5606813
:107720001F210902884329690902084360600FE0AC
:107730002068400840002060FFF798FA064604E001
:10774000FFF794FA801B022896D820684007F7D4E8
:107750002878C00660D5002F0CD0A86900284AD030
:107760002068FF21013108432060FFF77FFA0646B9
:107770002EE0C1E02068800502D5A8690028A6D0C7
:107780006068072149038843296A0843606060688C
:10779000297F0002000A090608436060286A410B3D
:1077A0000120C003491C8840E16809060A0F91497D
:1077B000895CC8409049086090480068FFF778FAF3
:1077C000002817D128E0FFF751FA801B0228A2D821
:1077D00020688005F7D56068072149038843296A36
:1077E000084360606068297F0002000A09060843B8
:1077F000606011E0E2E02168FF20013081432160F8
:10780000FFF734FA064604E0FFF730FA801B02283F
:1078100072D820688005F7D42878794E000724D5DF
:1078200068690028306910D0012108433061FFF7F2
:107830001DFA009005E0FFF719FA0099401A022896
:107840005AD830698007F6D50FE040084000306113
:10785000FFF70CFA009005E0FFF708FA0099401ACC
:10786000022849D830698007F6D42878400766D5C1
:1078700000200290A06BC00006D4A06B0121090774
:107880000843A063012002905E480168C90511D435
:107890000168821511430160FFF7E8F9009005E0E7
:1078A000FFF7E4F90099401A642825D85548006884
:1078B000C005F5D5FF20AA680130824203D13169A5
:1078C0000143316111E001218902002A07D005231B
:1078D0001B029A4203D132690A433261EFE73269EF
:1078E00082433261306988433061A868002810D033
:1078F000FFF7BCF9009008E05FE0FFF7B7F9014639
:107900000098091A4048814257D830698005F4D55B
:107910000DE0FFF7ABF9009006E0FFF7A7F900993B
:10792000411A3948814248D830698005F5D4029817
:10793000002804D0A06B012109078843A063686A6E
:10794000002866D00C2F3ED001263606022820687B
:1079500005D0B0432060FFF789F905462FE0B0431A
:107960002060FFF783F9074604E0FFF77FF9C01BAB
:10797000022822D820688001F7D4E96AA86AE26860
:107980000843296BFD231B049A4311430843E0601D
:10799000206830432060FFF769F9054604E0FFF7EF
:1079A00065F9401B022808D820688001F7D530E02F
:1079B000FFF75CF9401B022801D90320FEBD2068B7
:1079C0008001F5D425E00128F8D0E0680121090400
:1079D000AA6A014091421AD10F218904EA6A014042
:1079E000914214D1032189050840296B88420DE09A
:1079F000001002405EC80008840100207C010020C5
:107A000040100240007000408813000001D00120A7
:107A1000FEBD0020FEBDF8B504000ED0FF27606A51
:107A20000537002500280AD02561656126464036C5
:107A3000A562707C002807D00AE00120F8BD6068CC
:107A4000B842F3D0E561F1E73574204600F03EF826
:107A5000022171742068026840239A430260212346
:107A6000A26860689B021A4038401043E3688A02AB
:107A70001340184323690B40217D1843C907C90FE0
:107A80000843A169931019400843E169382319405C
:107A90000843216A802319400843A16A93001940D2
:107AA000084321680860A0690421000C0840616A4D
:107AB000102319400843216848602068C169914338
:107AC000C1616565012070740020F8BD10B586B0F5
:107AD000044614216846FDF76AFB10492068884275
:107AE00019D10F48416B821411434163C16A0122CD
:107AF0001143C162C06A002110400590E02000904F
:107B00000220019003200390029104910520694610
:107B10000007FEF7DBFF06B010BD0000003001409B
:107B200000100240094910B5401E884201D90120C9
:107B300010BD074C60610321081F02F0C3FE002046
:107B4000A06107202061002010BD0000FFFFFF00A2
:107B500000E000E0F0B502462032137E012B1ED07B
:107B6000012515760223537606687468B36870277A
:107B7000BC430F68274377600068AC07A04205D07C
:107B8000084CA04202D0084CA04204D1802449688D
:107B9000A34319438160557600201076F0BD022082
:107BA000F0BD0000000801400014014070B5050060
:107BB00005D02C462034607E002802D006E001204B
:107BC00070BD00202076284600F010F80220607674
:107BD000291D286802F09EF80120A077A076E076A3
:107BE000207760776076002070BD0000006801217A
:107BF0008907884204D10348816B012211438163C4
:107C00007047000000100240F8B5054604462035D4
:107C1000287E012817D001262E7602206876226859
:107C200090687727FF23B8431B02984390600A6847
:107C3000502A31D00EDC202A4BD006DC002A48D056
:107C4000102A3AD145E00220F8BD302A41D0402A1E
:107C500033D136E0602A27D0702A12D001200003E9
:107C6000121A2AD0824228D1CB684A6889682068D3
:107C700002F089F820688168012292031143816033
:107C80001BE0CB684A688968206802F07CF82168AC
:107C900088683843886010E0CA684968206802F044
:107CA000ECF85021206806E0CA684968206802F0B4
:107CB000F5F86021206802F071F86E7600202876D1
:107CC000F8BDCA684968206802F0D7F840212068EA
:107CD000F1E711462068EEE710B586B0044614219E
:107CE0006846FDF764FA012120688907884212D1AD
:107CF0000A49CA6A02200243CA62C96A0190014065
:107D0000059141020091002102910391049069467E
:107D10000348FEF7DBFE06B010BD00000010024075
:107D200000040050F8B5064604462036307E0D4665
:107D300001280BD0012008273076002A08D0042A19
:107D400016D0082A2AD00C2A4DD137E00220F8BDDF
:107D5000206802F02BF8206881693943816120682E
:107D6000816904229143816120688169EA6812E097
:107D7000206802F033F8206881690122D2021143A1
:107D8000816120688269012189028A4382612068B9
:107D90008169EA6812021143816124E0206802F0DF
:107DA00036F82068C1693943C1612068C16904227D
:107DB0009143C1612068C169EA6812E0206802F05D
:107DC00041F82068C1690122D2021143C1612068D3
:107DD000C269012189028A43C2612068C169EA68D7
:107DE00012021143C16100203076F8BD70B5050064
:107DF00005D02C462034607E002802D006E0012009
:107E000070BD00202076284600F00FF80220607632
:107E1000291D286801F07EFF0120A077A076E0767A
:107E2000207760776076002070BD704770B505469A
:107E30002C4602202034002908D004290BD0082920
:107E40000ED0627F012A10D0012070BDA27E012ACF
:107E5000FAD1A0760AE0E27E012AF5D1E07605E0CB
:107E6000227F012AF0D1207700E060770122286884
:107E700001F07CFF0122286892070121904205D081
:107E8000074A904202D0074A904204D182685207C2
:107E9000520F062A02D002680A430260002070BD19
:107EA000000801400014014070B504460D4600680A
:107EB000002201F05BFF2068016A0C4A114203D1E5
:107EC000016849084900016001202034002D06D0D6
:107ED000042D06D0082D06D06077002070BDA07656
:107EE000FBE7E076F9E72077F7E7000011110000E3
:107EF0007047704770470000F8B502680446D069C3
:107F000011689668814B05461D402023002D6CD0DA
:107F1000F7077F4DFF0FBC460D402F4379D0254614
:107F2000C7078035002F06D0CF0504D5012717627B
:107F30002A683A432A60820708D5F20706D02768E4
:107F400002223A622A6804273A432A60420708D587
:107F5000F20706D02668042232622A6802263243DB
:107F60002A6002070AD50A461A406646324305D0FF
:107F70002668082232622E6816432E60020508D554
:107F80004A0106D501222668D20232622A681A43C3
:107F90002A602A68002A30D0800606D5880604D5D3
:107FA000616E002901D020468847286821688968C9
:107FB000490602D42821084225D0204602F093F930
:107FC00020688168490619D5826840218A43826009
:107FD000206F002812D04F498163206FFEF7DCFB31
:107FE00000280AD0206F816B06E0850611D58D062A
:107FF0000FD5616E77E020468847F8BD2046FFF731
:1080000079FFF8BD05E02046FFF774FF00202860E7
:10801000F7E7256E012D56D1C50654D5CD0652D5AC
:1080200010261662206881682546490640350029D9
:108030002ADA226F116849680904090CE1D02F8BF4
:108040008F42DED9698311680968890617D40168EF
:1080500032019143016020688168490849008160CC
:1080600020688168402291438160E3670020206698
:1080700020680168B1430160206FFEF76BFB288B1D
:10808000698B401A81B21AE0298B6A8B891A6A8B34
:1080900089B2002AB5D00029B3D00268FF25213566
:1080A000AA43026020688268520852008260E36737
:1080B00000202066606620680268B24302602046A5
:1080C000FFF716FF9DE7C50208D5750206D501200A
:1080D000000510622046FFF70CFF92E7050605D564
:1080E0000D0603D5A16E002985D18AE7400688D503
:1080F000480686D5116820464024A1431160836755
:108100000021816600F043F97BE700000F080000C2
:10811000200100040DA2000810B5040003D0A06FD8
:10812000002802D007E0012010BD00217420015575
:10813000204600F027F82420A0672068016849083D
:1081400049000160204602F021F90128ECD0606A64
:10815000002802D0204601F043FF20684168092230
:10816000D20291434160206881682A229143816054
:1081700020680168012211430160204601F096FF4A
:1081800010BD0000F0B587B0064614216846FDF723
:108190000EF82C493068884251D12B48416B01229E
:1081A000920311434163C16A01221143C162C06A53
:1081B0000025104005900320400200900220032774
:1081C00001A9A1C104200490052069460007FEF71B
:1081D0007DFC1F4C1D48A560E56081C48027E560DB
:1081E000A7602020256160610002A0611848083C5A
:1081F000FEF74CFB002801D0FDF7FEFD3467A662B8
:10820000144C12482146143820600320606010206E
:108210000831A1C16561A561E56120462562FEF7CF
:1082200035FB002801D0FDF7E7FDF46600220121AF
:108230001B20A662FEF7A2FF1B20FEF793FF07B0EC
:10824000F0BD000000380140001002403000024044
:10825000501700209817002070B5C36F202B27D12E
:1082600000290BD0002A09D0012483682403A342EB
:1082700006D10369002B03D1CB0701D0012070BDCB
:10828000034660331C7D012C12D001241C75002391
:108290000366084C0368A34207D05C68240204D537
:1082A0001C680125AD062C431C6002F06FF970BDFF
:1082B000022070BD0048004070477047FFB504467B
:1082C000806F83B017460D4620285ED1002D0AD05E
:1082D000002F08D0A168C001814207D12069002881
:1082E00004D1E80702D0012007B0F0BD204660307D
:1082F0000090007D012848D00098012101750020E0
:10830000802108512120A067FEF7B0FC26464036A8
:108310000190378277820120A1680003814202D157
:108320002069002805D02F460025009900200875F7
:1083300011E00027F9E700228021204602F06CF9C5
:10834000002815D1002F15D02168387888627F1C4D
:10835000708A401E7082708A019B002806980090E7
:10836000E9D100224021204602F056F9002808D029
:108370000320B9E728882168C005C00D8862AD1CBC
:10838000E6E72020A0670020AEE70220ACE77047B8
:10839000034D044C04A002F039FAE560FAE700004E
:1083A0000400FA0500ED00E0486172644661756CF6
:1083B000745F48616E646C65722E0D0A00000000E7
:1083C00000B585B014216846FCF7F1FE0348022190
:1083D000418300F0FFFB05B000BD00003C01002020
:1083E00010B505242407002204212046FEF737FC9F
:1083F000002208212046FEF732FC0A2002F06BFC26
:10840000012204212046FEF72AFC0A2002F063FC28
:10841000002204212046FEF722FC10BD10B50524E1
:108420002407002204212046FEF719FC012208211E
:108430002046FEF714FC0A2002F04DFC0122042124
:108440002046FEF70CFC0A2002F045FC0022042125
:108450002046FEF704FC10BDF8B5002405260746AB
:1084600025463607002204213046FEF7F8FB0A2095
:1084700002F031FC012204213046FEF7F0FB6006D9
:10848000040E08213046FEF7DDFB002801D0641CF5
:10849000E4B2052002F01FFC6D1CEDB2082DE1D303
:1084A000002F03D0FFF79CFF2046F8BDFFF7B6FF73
:1084B000FAE770B505260546360700220421304646
:1084C000FEF7CDFB0024E80901D0012200E00022E4
:1084D00008213046FEF7C3FB6806050E0A2002F0AD
:1084E000FAFB012204213046FEF7B9FB0A2002F014
:1084F000F2FB002204213046FEF7B1FB0A2002F015
:10850000EAFB641CE4B2082CDDD370BD10B5052471
:108510002407012208212046FEF7A1FB01220421A5
:108520002046FEF79CFB002208212046FEF797FB21
:108530000A2002F0D0FB002204212046FEF78FFB28
:1085400010BD10B505242407002204212046FEF7A3
:1085500086FB002208212046FEF781FB0A2002F05C
:10856000BAFB012204212046FEF779FB01220821F3
:108570002046FEF774FB0A2002F0ADFB10BD70B57B
:1085800005252D070024012208212846FEF767FB58
:10859000062002F0A0FB012204212846FEF75FFB23
:1085A000062002F098FB07E0641CE4B2FA2C03D921
:1085B000FFF7C7FF012070BD08212846FEF742FBE8
:1085C0000028F1D1002204212846FEF748FB0020B4
:1085D00070BD0000F8B501F09BFD01F0CBFD5B48DC
:1085E0000068C069FDF7F8FC594C5A49A082898F90
:1085F000594E0025002931D0A26A730357499A4287
:1086000002DB02220A7000E00D700A780121890263
:10861000002A05D0012A0ED0022A10D0032A1DD12B
:10862000608B01282ED0022818D1484808214038F4
:10863000FFF73AFC12E0FF22F5329042F0D2608B55
:1086400001281DD0022804D008E03046FEF707FBC1
:1086500004E03E4808214038FFF7E8FBFDF7C6FD7F
:1086600020700121C9023046FEF7ECFA0127FF0312
:1086700000282DD03A480560A079002804D007E0F2
:108680000022E2E70122E0E70120A07102F026F8D3
:1086900080213046FEF7D6FA002806D000220821B5
:1086A0003046FEF7DCFA012205E0012208213046BF
:1086B000FEF7D5FA0022052039460007FEF7CFFA6B
:1086C000244C284E4034A08C274F012803D01CE0B6
:1086D000A5710022EAE725486946088072B6802124
:1086E0002348FDF7A1FB002804D002226946204858
:1086F000FDF73EFC62B61FA002F088F8A58403F0E7
:10870000C1FF642002F0E0FAFE60608C012808D10D
:1087100010486584058003F0B5FF642002F0D4FAA8
:10872000FE60208C012806D1258403F0ABFF642075
:1087300002F0CAFAFE600748124A0188914202D14B
:10874000C088002800D1FE60F8BD0000CC160020D3
:108750003C010020E80D00200004005081000020B2
:10876000740100200400FA0500ED00E0AAAA000050
:10877000384A0008BDF8C8EBC9FDBCB6C4A3CABDE1
:108780000D0A0000AA55000038B55721202000F03E
:108790007AF80321212000F076F84021222000F011
:1087A00072F80821232000F06EF8AA21302000F092
:1087B0006AF81048018F142901D8002901D101213C
:1087C00001870C4C40346188142901D8002901D15B
:1087D00002216180008FC1B2322000F054F8A178EC
:1087E000332000F050F8684600F006F80A2002F046
:1087F00072FA38BDE80D002010B501460F2000F0D8
:1088000021F8002800D0012010BD10B50446FFF764
:108810007DFE3220FFF74DFEFFF7B1FEE0B2FFF71D
:1088200048FEFFF7ACFEFFF771FE3320FFF741FE75
:10883000FFF7A5FE0020FFF70FFE0446FFF781FEBD
:10884000204610BD10B50C46FFF7DFFF2070012059
:1088500010BD70B50D460446FFF758FE3220FFF7F5
:1088600028FEFFF78CFEE0B2FFF723FEFFF787FE3E
:108870002846FFF71EFEFFF782FEFFF762FE0A2082
:1088800002F029FA70BD10B5FFF7E3FF012010BD1B
:1088900010B50248FEF725FB10BD000004160020AD
:1088A000FEB50446002772B6334A01688B1804D11E
:1088B0003248C76803208004074088680190C86870
:1088C000009048698E69002B08D12C4940398B6A89
:1088D000CD042B438B628B6AAB438B6201463143E1
:1088E0003CD025492368CB4205D12449CA680323DB
:1088F0009B049A43CA6025462035002810D0216881
:108900000A6901231A430A61216848610821204647
:1089100000F036F8032800D1A873216808204860C9
:10892000002E10D0206801690122114301612068E6
:1089300086611021204600F023F8032800D1A87397
:108940002168102048600C482168C14206D10B48BC
:10895000C1680322920491433943C16020680169D0
:1089600049084900016121680198886021680098E0
:10897000C86062B6FEBD00000084FFBF4010024028
:1089800070B506460B480D46002409490068FCF7FF
:10899000AFFB7D21C90048433168401E00D103244C
:1089A0000B682A469A4301D00028F6D1204670BDB4
:1089B000204E0000840100201CB5002116480091C3
:1089C000144A01910260C16312054260816007226E
:1089D0008263012202610246C16020321170FF23CE
:1089E0005170C23343628162117301638161042259
:1089F00041634261C161FDF713FD08480090801397
:108A0000019069460448FDF7BBFC00210248FDF7D0
:108A100061FC1CBD00240140A815002002000004D8
:108A200008B50848016B012211430163006B012165
:108A30001040009000220A20FEF7A0FB0A20FEF75B
:108A400091FB08BD00100240F0B587B014216846C4
:108A5000FCF7ADFB4748C26A04210A43C262C26AFE
:108A60000A400592C16A80263143C162C16A314021
:108A70000591C16A01242143C162C16A2140059167
:108A8000C16A02252943C162C06A22462840059076
:108A900005201C210007FEF7E2F80122364937487D
:108AA000FEF7DDF8002236493448FEF7D8F8912168
:108AB0000520002209020007FEF7D1F83148019095
:108AC000002705206946029700940007FDF7FEFF86
:108AD0000C200090112001900320039005200297A4
:108AE00069460007FDF7F2FF10206A46039591C220
:108AF000052069460007FDF7E9FF11200190029764
:108B00006946039700941D48FDF7E0FF1E48019059
:108B10006946009502941948FDF7D8FFE0020090DD
:108B20006946019702951548FDF7D0FF1748694639
:108B300091C1694611480397FDF7C8FF91200002D3
:108B4000694691C10520694600070397FDF7BEFFFE
:108B500069460A48019700960294FDF7B7FF002284
:108B600001210520FEF70AFB0520FEF7FBFA07B0FE
:108B7000F0BD00000010024001020000000400509F
:108B80000830000000001110000021100832000021
:108B900010B50F4C0D482060FF20053060600020AC
:108BA000A060E06020616061E06101212062490213
:108BB0006062A161A0620720E0622046FEF72BFF01
:108BC0002068016840221143016010BD003001405F
:108BD0003416002010B58AB000240494059406943D
:108BE0000794089401211848099400940194029470
:108BF000890703940160092184604160046113497D
:108C00004461C160FEF7D2FF01200003049004A973
:108C10000D48FEF7F9FF0C48FFF7E8F8089408A99B
:108C200009480994FEF796FF6020009008480190DB
:108C300002940822694603940348FFF773F8024838
:108C4000FFF74AF80AB010BD8C160020930400000C
:108C50005702000000B585B014216846FCF7A7FA5A
:108C60000E480D490160E121490241600021816007
:108C7000C160016181610C22C161426101623021E8
:108C800041620121090381634900C163FFF744FA8E
:108C900001F01EFD05B000BD00380140CC160020DB
:108CA00070470000F0B589B00A2002F05FFD7D201A
:108CB000400102F075FDFF4C0025A570FE48E065FF
:108CC000A07B0C2801D30B20A07360790A2801D95E
:108CD0000A206071F948E570F94E00783071F94961
:108CE000A079097840000843E17C89000843F071CD
:108CF000A06BF070010A3172401CA0636079B074FF
:108D000042003046F0491330FCF738FA6079EE49FA
:108D100082004000801960311330121DFCF72EFADA
:108D200060790621420048438019E8491730921CB7
:108D3000FCF724FA2C20205E002803D0E449098A9D
:108D40000818A0856079DB49C000203182190B7BAF
:108D500053764B7B937606227272DE4A1D30127870
:108D6000B272628C3273D64A0B79133A1375497911
:108D700051750022D24902F0E3FD60790021C00064
:108D80001D3002F0EFFDD448FEF786F90127E0849C
:108D9000BF0309E0D048FEF77FF980B2E084A18EDE
:108DA000FF392D39884206DBA18E80B28842F1D38B
:108DB000C9198842EED8022002F028FDC0480126D9
:108DC000C571E573E57266732573C348FEF764F9F0
:108DD00020850746E5706079FCF7B0FCBF4AC04BC0
:108DE000FCF790FB01F00CFF0022BE4BFCF7D8FA19
:108DF000FCF704FD0006C10CC81980B2F1036085C0
:108E0000884201D3401A6085B748A0642079401C8D
:108E10002071B148FEF740F9E084AB48A54F6438B3
:108E200040370690B1E1AC48FEF736F9E0840BE03C
:108E3000A948FEF731F980B2E084618D884203D3FE
:108E4000AA4A8918884207D300210F2002F00EFC9D
:108E5000A749E0630842EBD0E06B411C1FD04004FF
:108E60007ED58122D20100210F2002F03EFD00219B
:108E7000102002F0FBFB41069348490E00227C388B
:108E8000A16502F029FC002002F08AFC002002F01B
:108E90003CFC8D487C38417A0729C3D101E001F0C0
:108EA00033FD02229349401DFCF78CF90028B9D10B
:108EB00002F0A9FDE167A06702F092FD7D4B8033CF
:108EC00003C3E0788049401CE07083390B7A684620
:108ED0000370497A417000880390A18C88427DD14B
:108EE000774985488C31C98E0180754971488C312C
:108EF000098F01847848FEF7CFF8E08402F0C8FAC1
:108F00006C48FF22803001684068520400238918B1
:108F100058410206080A10434108490000900A0E11
:108F2000080264498031CA6088606548E36F0A308E
:108F3000A26F02F03DFD60798100614808185D492B
:108F4000163080310CC902F033FD5A488030C368B6
:108F500082685B48123002F02BFD0821584800E07F
:108F600006E14172B430C07C0009A07414D05648A8
:108F7000022260497738FCF725F900280CD15048C7
:108F8000E673C671A06D50491638C2B26639C81D65
:108F90002274FB30FCF7F2F8607900228000484927
:108FA0001C3002F0CDFC6079002180001C3002F002
:108FB000D9FC009802F0D3FB012002F027FC60727C
:108FC00002214E48FDF73EFE00281DD000213D48FD
:108FD00001703B498C31488E049000E05AE0B88023
:108FE000888EF8808446606CFF310531A06408608B
:108FF000DC39E064C97C0907090F032900D06174DA
:10900000A16D1C2902D015E00121E0E72C49294A75
:109010008C31C98FD185069B2C4A1B8813808842CE
:1090200007DD002805DD002903D0607D401C607548
:1090300000E065752571E672049838816046788194
:109040002673208C2E49FF30C33080B220848842A2
:109050000CD949424018208427487D220188D2003B
:10906000491C89B20180914200D3058022487D21AC
:109070000088C9004843218C4018206500F070FD2D
:10908000607A002805D100210F2002F0EFFA0006D7
:10909000F9D583E0FCF788FF0B4A03219032115485
:1090A00007498C314A8EBA80898EF980A26D1C2ABC
:1090B0002ED127E0700000203F420F003C0100202D
:1090C0005C120020700100208C130020C8140020C6
:1090D000280E00204C01002004160020B81E85EB4D
:1090E00051B8CE3F00000840A0860100983A000029
:1090F00000D02724600100206C01002000040050F3
:10910000E70300005F4B4200D318069A12885A808A
:1091100080005D4B5C4AD43B02905B4982189B8F78
:10912000138030314118626C4A60584940185849E0
:1091300016300CC902F03CFCE16D606C884207DA25
:10914000514A02995158012902D1E06503990591CC
:109150004D49029A8958814217DD012915DD2246C1
:10916000002812DD0398908402201070A5720CE094
:10917000484A00210F2002F0B8FB6079E178401CDA
:10918000814202D0002002F0C0FAE18C608D814261
:1091900000D248E6404A80188142FAD8E07A012895
:1091A00001D00220E07202F073F93A4A00210F2048
:1091B00002F09BFB2179002914D0384800888200F6
:1091C00082188A4200D22570002000F0E1F8E07B8E
:1091D000002836D02C496C310B7848788A78022BDD
:1091E00017D02EE0A16CE26D323920468A420EDAA9
:1091F000C1792A4A491CC9B2C171128852008A42F7
:10920000E5D20599818402210170A572DFE7E5713D
:10921000DDE710280CD0C82813D2214BC91C181820
:10922000FBF7ACFF03F02EFA642001F04DFD36E6AB
:109230001C4D28684000000E03D1C878FCF763FA83
:10924000286000202378A27A65790FE00E4E410055
:10925000303E775A1836765AB74205D00A4F022365
:1092600000220126483F7E52401CC0B2A842EDD3E6
:109270002370A272074A002180320F2002F035FBD2
:1092800009B0F0BDC8140020BC1300205C120020FF
:10929000F000002000D02724983A00004C01002064
:1092A000E80D002064010020F8B52E4C0546A06EA4
:1092B0002D4A281A411EE066914215D21821615E9E
:1092C000081AFCF727FA294A294BFCF71BF906462E
:1092D00030200F46205EFCF71DFA32463B46FCF775
:1092E0005FF8FCF767FA20860020A0751D481A2356
:1092F000C35E428C1F48008884461F4806881DE0D4
:109300006046484380181D4F80B23880302778432C
:109310006427643078431A4F2066C01985420BD207
:10932000C8B2184930220880206EA25E411BC918BD
:1093300089186166A066F8BD491CA175A17DB1427E
:10934000DED33020424310486421101848430F49AF
:109350004118A16620663021401B615EC01840188C
:109360006066F8BD70000020CF0700009A999999B7
:109370009999B93F5A0100204C0100206E0100204C
:1093800078ECFFFF5801002074270000C0BDF0FFFB
:10939000FEB5294D2988491C8FB228492F800E8897
:1093A000FCF7B8F9264A274BFCF7ACF8019100907E
:1093B00025483146FBF79CFE244CE18E4218B7420B
:1093C00006D3002028802248019E1018009D02E04C
:1093D0001046019E009DFCF7B1F933462A46FBF783
:1093E000DFFFFCF70BFA6086012580B2ED03A8428F
:1093F00001D3401B6086A08BFCF7A0F9154A164BE1
:10940000FCF7E8F80646608E0F460090FCF796F9E8
:1094100032463B46FBF7C4FFFCF7F0F980B2A0866A
:10942000A84201D3401BA0860C49009809684861F6
:109430000098E086FEBD0000580100204C0100208D
:109440001904560E2D624040E17A000070000020A1
:109450001F050000F853E3A59B843E40041600203E
:1094600070470000F0B589B0002004900A2002F097
:109470007DF97D20400102F093F9B348002282700B
:10948000816BB34C491C8163B049838D098A2546A1
:10949000C91881852146027513310791473103911F
:1094A0006D393135AB4F203005910290A64E0F211A
:1094B000A948717100782071A84AB07912784000EB
:1094C0001043F27C92001043E071308FE070000A8C
:1094D0002072A17431461E229C310798FBF74EFE84
:1094E000402228469E49FBF749FE029903980A7BD1
:1094F000C274497B0175092060729A480078A07295
:10950000708C2073307D410030469C3009180598DE
:109510000A78027549784175762000228C4902F05C
:109520000FFA70790621484300211C3002F01AFA24
:10953000022002F06BF900210F2002F097F8384268
:10954000F063F8D0F06B411C18D040047ED5812226
:10955000D20100210F2002F0C8F90021102002F0F2
:1095600085F841067A48490E0022B43002F0B4F87A
:109570007748B430417A022902D0BDE001F0C4F945
:1095800002227949401DFBF71DFE0028F5D16E48E7
:109590000222007D41006C489C3009186C48B530AF
:1095A000FBF710FE0028E8D102F02DFA664AD167D9
:1095B000906702F015FA644A803203C204980028CA
:1095C0002CD1012004906248684E8C30C08E6049D6
:1095D00030805D488C31098F01846548FDF75CFD62
:1095E0005949644AC884088CFF30C33080B208846B
:1095F00090420CD952428018088430885D4A401C41
:1096000080B20B323080904201D30020308030880D
:109610007D22D20050430A8C801808654C48694668
:109620008C30428E0A80808E488049490422B531B0
:10963000C81FFF38FBF7A2FD4348494A007D009947
:10964000800011504049803103C900E075E0FF23DC
:109650005B040022C01851410906060A0E43304639
:1096600002F07DF8710849000A0E0802364900260A
:109670008031CA6088603448C36F826F344848388C
:1096800002F096F9304880300CC83148443802F076
:109690008FF92D488030C36882682D48403802F029
:1096A00087F92B49002252393C2002F049F9002168
:1096B0003C2002F057F9012002F0A8F82249487234
:1096C00008468078401C887001210520C9030007E6
:1096D000FCF77EFC1C48407A002805D100210F20B1
:1096E00001F0C4FF0006F9D5802200210F2002F00E
:1096F000FCF81548467002E01349012048701248F2
:10970000017D491CC9B201750F2900D2CEE604982B
:10971000002810D10C4A1849508C002802D00B8820
:10972000984201D908885084144980B20988401EA3
:1097300048431349088009B0F0BD124A00210F20A8
:1097400002F0D3F8D8E7000070000020280E0020B7
:109750005C12002000D027243C0100207001002072
:10976000781400204C010020600100206C010020D2
:1097700004160020E70300004801002046010020F5
:109780004401002000902724F8B531492F48086093
:1097900002F01CFA2F4800F0A3F92F4CE0822D486C
:1097A000801C00F09DF920832A48001D00F098F9E4
:1097B00060832B4829494180014640310979294F6E
:1097C0000906090E617006D1C7800121C1870A21EF
:1097D000418700218187244AC18E1170C18F217178
:1097E000818F6171817AA1708588052165626181AF
:1097F000C6883046FBF77CFCA08101462846FBF773
:1098000077FC8800081885B2164825816843FBF765
:1098100095FF164A164BFBF7DDFEFBF7EFFFE081E5
:10982000658231463846FBF763FC20820146C8203A
:10983000FBF75EFCE0830120A083FCF7CDFBA08258
:10984000E2890C490C48FDF72BFCF8BDFDA6000889
:1098500068000020004F00083C0100202B0200009F
:10986000E80D0020E803000018000020F853E3A5ED
:109870009B843E40FF7F000004160020F8B5754C25
:1098800000202071744D01202880744EC820308043
:10989000207A401C2072C00706D0608C411E618473
:1098A000022801D2C82060840120C043FFF770FD68
:1098B0000A2001F05BFF7D20400101F071FF0221D1
:1098C0006748FDF7BFF900283FD0002065498000B8
:1098D0000978664F49000843634909780843B8721C
:1098E000102078726248C1887D20C000FBF700FC20
:1098F000787360485E490078B87338460B308A78D0
:109900000270C97841705A49421C20310B7ED370D5
:10991000497E11715649D01C22310B7E5371497E0C
:109920009171534940310A7C0271497C4171002296
:109930003946172002F004F80021172002F012F82F
:10994000022001F063FF4C4F03E00120BEE7FEF769
:1099500041FE00210F2001F089FE3842E063F6D07D
:10996000E06B411C73D040046FD58122D2010021ED
:109970000F2001F0BAFF0021102001F077FE410610
:109980003A48490E0022B430A16501F0A5FE374FD8
:10999000B437787A112858D102223849781DFBF75C
:1099A00011FC002851D1F81F027A69460A70407AEA
:1099B0004870B97A2980C820FBF79AFB3080387B41
:1099C000608438462E4D2838C08E2880394621487C
:1099D0002839098F01842B48FDF75EFBE084208C39
:1099E0002949FF30C33080B2208488420CD94942D3
:1099F0004018208428882449401C80B20B312880DC
:109A0000884201D30020288028887D21C90048434E
:109A1000218C4018206500F0A3F868460088A084D7
:109A20001249B87CC7316071420008460D46693062
:109A3000FBF7A4FB6079294642001448FBF79EFB24
:109A4000608CFF2801D003202070F8BDFFE700F0F4
:109A50005BFF0000700000204C0100205A01002034
:109A60000004005040010020410100205C12002051
:109A7000E80D00201800002000D0272460010020FD
:109A80006C01002004160020E7030000A41300204E
:109A900070B586B014216846FBF789FB01250F4E8F
:109AA000ED03002229463046FDF7D9F801200024B5
:109AB000019002946946009503943046FDF706F83C
:109AC0000320019002946946009503943046FCF708
:109AD000FDFF022001F0F8F806B070BD0004005050
:109AE0000088704770470000F8B5044600206A46B9
:109AF0001080194D55222A70AA226A700322AA707A
:109B0000661DEE702A716971144A49008918AC719A
:109B10002246E81DFBF732FB002007E029186A46C1
:109B20008978128889186A461180401CB042F5DB9A
:109B3000611DA81CFCF7AEF8014668460180291992
:109B40000078C87168464078087221460931024899
:109B500000F0EAFBF8BD000042150020E80D0020EF
:109B6000FEB5FFF7A1FB2548FDF796FA244C86B217
:109B7000E68460790A21081AC000FBF7CBFD07468E
:109B80000191606EFBF7DAFD1E4A1F4BFBF722FDC9
:109B900000900D463046FBF7D1FD2B46009AFBF7AF
:109BA000FFFB3A46019BFBF7FBFBFBF727FE85B269
:109BB0006586A08BFBF7C2FD124A134BFBF70AFD2B
:109BC00006460F462846FBF7B9FD32463B46FBF7F3
:109BD000E7FBFBF713FE81B20120C003A18681429F
:109BE00001D3091AA186854201D3281A6086034948
:109BF000608E09684861E086FEBD00000416002002
:109C000070000020F853E3A59B843E40034A11688E
:109C1000382389B2994301431160704700300140F5
:109C200010B5FDF729F810BD10B59AB0342168467B
:109C3000FBF7BDFA14210DA8FBF7B9FA1C2112A8F5
:109C4000FBF7B5FA1B4801680324E402A143C214E0
:109C500089180160FDF79EFA17480169A143016167
:109C600006200090FF200130029001200390102078
:109C700004900220099040040B90000100240C90F5
:109C80000A946846FDF7B4FC0F200D9003200E9057
:109C90000F941094012111940DA8FDF77FFB8120F2
:109CA0001290032080041890149412A8FDF7C4FAAF
:109CB0001AB010BD0070004040100240104801680A
:109CC000821511430160C1680E4A1140C1600168EC
:109CD0000D4A1140016081684908490081600168AE
:109CE0000122920491430160C168FD221204914354
:109CF000C160002101610649044888607047000086
:109D0000001002400C40FF88F6FFF6FE00500008ED
:109D100000ED00E070B5026801239B07114C124D65
:109D2000984203D0A04201D0A84203D17026B2438A
:109D30004E683243984203D0A04201D0A84204D1D9
:109D400003231B029A43CB681A4380239A430B696F
:109D50001A4302608A68C262096881620121416116
:109D600070BD0000000801400014014010B5CB0692
:109D7000DB0E0121046A99408C430462016A9A4017
:109D80001143016210BD30B58468FF252D021B020E
:109D90001343AC430B432343836030BD826870237D
:109DA0009A430A4307210A438260704730B5026A2A
:109DB000520852000262026A456883697024A34314
:109DC0009C080B68A40023430224A2438C684560CE
:109DD0001443836149684163046230BD30B5026A4F
:109DE00010239A430262036A45688269732424023D
:109DF000A2430C6824021443202293438A684560DE
:109E000012011A43846149688163026230BD30B532
:109E1000026AFF2301339A430262026A4568C369FA
:109E20007024A3439C080B68A4002343012464020C
:109E3000A2438C68456024021443C3614968C1632E
:109E4000046230BD30B5026A01231B039A430262EB
:109E5000036A4568C26973242402A2430C68240281
:109E600014430122520393438A68456012031A4344
:109E7000C46149680164026230BD30B5036A046A96
:109E80006408640004628469F025AC431201224333
:109E90000A24A3430B438261036230BD30B5036AD9
:109EA0001024A34303628469036A0F252D03120360
:109EB000AC432243A024A3430901194382610162F8
:109EC00030BD0000F8B5102405252D07AC62AF2089
:109ED000800000F000FFAC6101F0DCFB344C354F3A
:109EE000354E20670EE001F0D5FB2067FEF772FBD0
:109EF000206C411C2164142804D930A000F086FC99
:109F00003248C760206FB042EDD100262664207829
:109F10000127FF03030000F0B2FC05040C192D3AE1
:109F20003C00012239462846FCF799FEFFF7A6FCC3
:109F300006E0012239462846FCF791FEFFF792FA27
:109F4000002239462846FCF78AFE22E0A07A012248
:109F5000401CA07239462846FCF781FEFCF758F8F1
:109F6000002239462846FCF77AFEA07A052810D947
:109F700026700EE0FEF796FEFCF7ECF81548144943
:109F80000068FBF785F9FBF7E7FBA08501E0FFF729
:109F900069FA02211048FCF755FE002805D0002080
:109FA0000E49087001F05CFAF8BD0120F8E70000E6
:109FB000700000200400FA053001CADE4457204931
:109FC00044204552524F522E0D0A000000ED00E091
:109FD0000000C84200000020000400507001002072
:109FE00010B5818CC90707D001684A6801235B045A
:109FF0009A43836A1A434A60818C890707D50168AE
:10A000004A6801231B049A43C36A1A434A60818C3D
:10A01000490707D501684A6801239B049A43036BEB
:10A020001A434A60818C090707D501684A680123F1
:10A03000DB039A43436B1A434A60818CC90607D5F8
:10A040000268916801231B039943836B1943916054
:10A05000818C890607D501688A6801235B039A43CE
:10A06000C36B1A438A60818C490612D503685A680B
:10A0700001210905046C8A4322435A60026C8A421A
:10A0800007D10268516803235B059943436C194368
:10A090005160818C090607D501684A680123DB04F9
:10A0A000806C9A4302434A6010BD0000F8B5044634
:10A0B000002680300660FCF7D9FD05462068006860
:10A0C000124F000709D501212B46002249052046E1
:10A0D000009700F0A1FA00280DD120680068400721
:10A0E0000BD501212B46002289052046009700F060
:10A0F00093FA002801D00320F8BD2020A067E06774
:10A100002666603426750020F8BD0000FFFFFF01C1
:10A11000F8B5154CC826E078002823D160790028CE
:10A1200020D101206071114D686B0027002818D0E4
:10A13000686BC821081A0FE00D48E168405C61694E
:10A140008847E068401CE060E068C82800DBE76002
:10A15000696BC820401A761EE168814201D0002E4A
:10A16000EADC6771F8BD00005400002000000240E6
:10A17000200D002070B5224CE07800283FD12079D6
:10A1800000283CD1012020711E4EF16900250906EE
:10A19000002933DA2156625791420AD1F06940060C
:10A1A0002CD5A079002829D0A5712089401C2081B8
:10A1B00024E0A179002903D1A0710A2000F08BFDD1
:10A1C00000202056CC2148430F494218206912181C
:10A1D0001279B262401C00222061A256CC235A435D
:10A1E000895881420ADC25612078401C2070207843
:10A1F0000E2800D12570A078401CA070257170BD7C
:10A200005400002000380140F801002010B5806A99
:10A210000022014640314A834A82FDF76BFE10BDA1
:10A2200070B5846AA06FE56F216889680026090609
:10A23000002906DA212804D152200653204600F0D6
:10A240006BF820688068400606D5222D04D15A207C
:10A250000653204600F047F820468030016810225F
:10A26000114301602046FDF745FE70BD10B5014663
:10A270000968806A096889061CD400225A210A529A
:10A2800001680A68FF2301339A430A6001688A68FB
:10A29000520852008A6001688A6840239A438A60A3
:10A2A0002021C167016E012904D101680A681023C9
:10A2B0009A430A60016E012902D0FDF7FDFF10BD2F
:10A2C0005821095AFDF714FE10BD10B5806A016EC1
:10A2D000012902D0FDF7F1FF10BD5821095A4908A4
:10A2E000FDF706FE10BD01680A68FF2321339A437B
:10A2F0000A6001688A68520852008A60016E01296A
:10A3000004D101680A6810239A430A602021C167BA
:10A31000002101664166704701680A68C0239A43BC
:10A320000A6020218167704770B5164CE278002AD8
:10A330000CD12279002A09D10122E2700025C82916
:10A3400003DC0222A256002A01DCE57070BD012365
:10A35000E356CC2253430C4AD1500123E356CC267A
:10A3600073439B180A460146181DFAF707FF6078E9
:10A37000401C607060780E2800D16570A078401E87
:10A38000A070E2E754000020F8010020F8B5044670
:10A39000016880682369E6691843636900253343CF
:10A3A0001843724A0B68724E334003430B602168B6
:10A3B000486803231B039843E368184348602168F7
:10A3C000A069914201D0236A18438B680B2636029C
:10A3D000B34303438B606749236867488B420CD1C2
:10A3E000C0688007800F06D0012839D0022835D0F8
:10A3F000032821D11EE001271FE060498B420AD1CA
:10A40000C0680C21084027D0042829D0082825D06E
:10A410000C2811D10EE093420ED1C16803208002B6
:10A42000014019D001208002091A19D0091A15D04B
:10A43000814201D1082700E010274F495048403998
:10A440008600934232D1002F0CD0022F0DD0042F62
:10A4500010D0082F7FD126E00027EEE70227ECE797
:10A460000427EAE7FDF768F806E00968C90605D49D
:10A47000304603E0FDF780F8002872D06268510092
:10A480005118814267D81103814264D3010E06023C
:10A490005008002330185941FAF740FE0321090201
:10A4A000411A384A55E00120C003E7E70122E36979
:10A4B000D20393422BD13B0000F0E1F90906090CCD
:10A4C0004D114D4D4D274D00FDF736F809E0FDF7D4
:10A4D00043F806E00968C90605D4304603E0FDF7F5
:10A4E0004BF800283DD0616840004A088018FAF710
:10A4F000FFFD80B20146244A103991422BD8511CED
:10A5000001400007400F084329E01046EBE73B00FD
:10A5100000F0B5F90906090C21122121212321009F
:10A52000FDF70AF80AE0FDF717F807E00968C90621
:10A5300006D4304604E00EE0FDF71EF8002810D0E7
:10A5400061684A081018FAF7D3FD80B201460E4A36
:10A550001039914203D9012503E01046F0E7216844
:10A56000C86000206066A0662846F8BD004800402C
:10A57000F369FFEF00380140401002400044004002
:10A5800000093D00FFFC0F00EFFF0000F8B5044696
:10A590004165403000262746028380373E602220F6
:10A5A000E0672546206F603500281CD01749C1623E
:10A5B000216F17480863216F16484863206F866330
:10A5C000236F606D9C461346216802466046243125
:10A5D000FCF7A4F9002806D0102038602E75202042
:10A5E000A0670120F8BD2E7520680168FF220132A6
:10A5F0001143016020688168012211438160206855
:10A6000081684022114381600020F8BD6DA20008DE
:10A61000CBA2000821A20008FFB581B005460F4675
:10A62000044660350A9E39E0701C37D0FCF71EFBEB
:10A630000499401AB04222D8002E20D02068016828
:10A6400049072BD5C069C043000527D401202168E4
:10A65000C002086220680168FF22A13291430160B4
:10A66000206881684908490081602020A067E06770
:10A670008034206000202875032005B0F0BD2068DC
:10A680000168FF22A1329143016020688168490876
:10A69000490081602020A067E067EBE72068C1697E
:10A6A0003846884305D0002103988142BCD0002061
:10A6B000E3E70121F8E7000010B50449102009681C
:10A6C00008620248FDF718FC10BD0000CC160020FF
:10A6D00001490D20887070475400002010B5FEF726
:10A6E0009FF9FEF7B7FAC82202490348FDF7B4FD07
:10A6F00010BD0000200D0020CC160020F8B53E4C07
:10A70000002321783D4A1D46082910D0072947D04B
:10A71000062950D0052952D0042953D0032954D0FA
:10A72000002956D0012958D002295AD05BE0A178DF
:10A7300000264A1F04E0314FBF5DFB189BB2761C18
:10A740009642F8DB667927799A195118E37862788E
:10A75000C9188918C9194018C0430006000E1AD13B
:10A76000012E14D0022E16D125482449C018FAF71C
:10A7700005FD01F087FF642000F0A6FABFF34F8FBC
:10A7800021492048C860BFF34F8F00BFFDE759083B
:10A790001046FFF7A9F92570E570A570A571F8BD01
:10A7A000A1795054491CC8B2A071A178491F8842B0
:10A7B000F5D1082001E0607007202070F8BDE0703E
:10A7C0000620FAE760710520F7E7A070E570042025
:10A7D000F3E7552807D10120EFE7AA2803D102208B
:10A7E000EBE7032803D02570E570A570F8BD0320C2
:10A7F00020702071F8BD000034010020DE1400201C
:10A80000E80D00200400FA0500ED00E010B5024A52
:10A81000024900F0E5F910BDC9B90008880100201F
:10A820002021020C01D010211046020A01D010464E
:10A830000839020901D01046091F820801D01046CC
:10A84000891E420801D0881E7047081A7047F8B563
:10A85000040C8BB2264682B25E430D0C1046370CB8
:10A860005843360480190021794116466E43370C4F
:10A8700036048019794126466E438919F8BD30B4F3
:10A880007446641E2578641CAB4200D21D46635D8D
:10A890005B00E31830BC18474900CA0202431000AD
:10A8A00000D004204A0D01D001221043044A490D72
:10A8B000914201D102210843012800D105207047AF
:10A8C000FF0700008307FF22DB0E9A408907090E6D
:10A8D0009940002808DB830809489B001B1818686A
:10A8E00090430843186070470007000F083883083A
:10A8F00004489B001B18D86990430843D8617047EF
:10A9000000E400E000ED00E0BFF34F8F044903488E
:10A91000C860BFF34F8F00BFFDE700000400FA05D9
:10A9200000ED00E0F8B504464F1EC80008382118B5
:10A9300015461E46086849683A4606239A4310D0D1
:10A940002A463346FAF7DEFD3A46D200083AA31803
:10A950001A687F1E5B68FAF723FD06223B46934385
:10A96000EED1022F23D0042F11D0062F2FD12A464B
:10A970003346FAF7C7FDE36AA26AFAF711FD2A46E1
:10A980003346FAF7BFFD636A226AFAF709FD2A46E1
:10A990003346FAF7B7FDE369A269FAF701FD2A46E3
:10A9A0003346FAF7AFFD63692269FAF7F9FC2A46E4
:10A9B0003346FAF7A7FDE368A268FAF7F1FC2A46E6
:10A9C0003346FAF79FFD63682268FAF7E9FCF8BDA1
:10A9D000002210B5134610460149FAF7FBFD10BDE1
:10A9E0000000F03F10B5FAF7DBFC10BD002210B5F7
:10A9F000134610461146FAF7EDFD10BD10B50721BC
:10AA0000024A00200907FAF75DFE10BD01030000AD
:10AA1000034A10B500201107FAF754FE10BD0000DC
:10AA200001FDFFFF02E008C8121F08C1002AFAD189
:10AA300070477047002001E001C1121F002AFBD1BE
:10AA40007047000001490860704700008C01002039
:10AA500008B50021684601706B46012202212C20B6
:10AA600000F052FF0221684601706B4601222C2043
:10AA700000F04AFF08BD000038B504466D20694665
:10AA800008706B46012207492E2000F03DFF064961
:10AA9000002C01D0054A00E0054A2E2000F01AFFE4
:10AAA00038BD000006080000061800000706000078
:10AAB0000716000038B504466B46022200213620F6
:10AAC00000F0EEFDB3212300FFF7D9FE0E0F0815AD
:10AAD0003A3A3A3A1C273A3A2F34483A0021684623
:10AAE000017040784108490014E069460878800800
:10AAF0008000401C04E06946087880088000801CC3
:10AB000008701DE0684602780A40483202704178B9
:10AB1000802001436846417012E0684602780A408E
:10AB2000027040784106490EF4E7694648780221F0
:10AB3000084303E069464878FD21084069464870AB
:10AB40006B4601220021362000F0DEFE012200AB20
:10AB500011463620013300F0D7FE38BD694608782B
:10AB6000CF21084069462030CAE708B5032168466E
:10AB70004170012101706B4602220021362000F055
:10AB8000C3FE0122D20306212D2000F0A3FE0120E6
:10AB900000F09AF80120FFF78DFF08BD08B5020A02
:10ABA00069464A7008706B46022204212D2000F08D
:10ABB000ABFE0320694608706B46012206212D205A
:10ABC00000F0A2FE0020694608706B4601220621B3
:10ABD0002D2000F099FE0A212D2000F047FD08BD30
:10ABE000F8B516460F460446002503E03946B0473F
:10ABF000641C6D1C20780028F8D12846F8BD0000A0
:10AC0000F8B54A002B4B520DD6182B4A0C46054678
:10AC1000142E2BDA002E12DA284BFAF7C1FB002291
:10AC20001346FAF731FE40D2002C03DA0124E40780
:10AC300000253AE02046284337D0214C14E0214F2C
:10AC40000B46F7403B402B4331D01C4BFAF7A8FB97
:10AC500000221346FAF718FE27D2002C03DD01204C
:10AC60000005F0400419BC4300251EE0332E1EDC15
:10AC700033460027143BFF43DF40384217D00F4BC9
:10AC8000FAF738FC00221346FAF7FEFD0DD2002C2D
:10AC90000ADD142E0CD03420811B0120884040197D
:10ACA000A84200D2641C0546BD4321462846F8BD93
:10ACB000641CF9E701FCFFFF9C7500883CE4377ECB
:10ACC0000000F03FFFFF0F007D2110B5C900484391
:10ACD00000F001F810BD002140E000BF00BF00BF40
:10ACE00000BF00BF00BF00BF00BF00BF00BF00BF6C
:10ACF00000BF00BF00BF00BF00BF00BF00BF00BF5C
:10AD000000BF00BF00BF00BF00BF00BF00BF00BF4B
:10AD100000BF00BF00BF00BF00BF00BF00BF00BF3B
:10AD200000BF00BF00BF00BF00BF00BF00BF00BF2B
:10AD300000BF00BF00BF00BF00BF00BF00BF00BF1B
:10AD400000BF00BF00BF00BF00BF00BF00BF00BF0B
:10AD500000BF00BF00BF00BF00BF491C8142BCD381
:10AD60007047FFB581B01E460F46040026D00B99F0
:10AD700003980143A06A394382680720904700285E
:10AD800018DB0A99A06A31438268062090470028A0
:10AD900010DB25462035A979032F01D9082001436E
:10ADA000032E01D904200143A06A8268092090473C
:10ADB000002806DA0120C04305B0F0BD0020C043E2
:10ADC000FAE7384600F000F92060304600F0FCF861
:10ADD00060600A9868700398A870EF702E710B98E5
:10ADE00068710020E8E70000F7B50446002090B045
:10ADF00000900190002C05D06A46062101F07CFCF1
:10AE0000062803DA0020C04313B0F0BD684640783E
:10AE1000010268460078000409186846807808181E
:10AE2000FAF78CFC054668460391007901026846F2
:10AE3000C07800040918684640790818FAF77EFCC3
:10AE4000032206460F4692075C4BFAF71DFD07D218
:10AE500000225B4B30463946FAF746FB06460F4662
:10AE600003229207554B28460399FAF70DFD07D2A6
:10AE70000022534B28460399FAF736FB0546039107
:10AE80002068FAF75BFC02460B4630463946FAF773
:10AE9000A1FB07460A200791205EFAF73BFC3A46E1
:10AEA000079BFAF72FFB064608200991205EFAF768
:10AEB0001FFC0021C943FAF766FAFAF7BDFC3246D7
:10AEC000099BFAF76DFA069108906068FAF736FC6C
:10AED00002460B4628460399FAF77CFB05461A20E2
:10AEE0000E46205EFAF716FC2A463346FAF70AFBAE
:10AEF0000C9009911620205EFAF70CFC099B0C9A25
:10AF0000FAF74EFA05910A902A46334638460799D1
:10AF1000FAF7F8FA059B0A9AFAF7F4FA05910A90FB
:10AF20001420205EFAF7F6FB3A46079BFAF7EAFA96
:10AF300007461C200791205EFAF7ECFB2A463346B1
:10AF4000FAF7E0FA0E900B911820205EFAF7E2FB78
:10AF50000B9B0E9AFAF724FA2A463346FAF7D2FAEE
:10AF60000B910E902069FAF7D5FB0B9B0E9AFAF71E
:10AF700017FA2A463346FAF7C5FA05460E46E06840
:10AF8000FAF7C8FB2A463346FAF70AFA3A46079B0D
:10AF9000FAF706FA059B0A9AFAF702FA01229207D3
:10AFA000084BFAF7AFFA02460B46129C089806992E
:10AFB00003C411980CC0002026E70000FFFF5F418A
:10AFC00000007041E17A843F00B50121C90403000B
:10AFD000FFF755FC081A05080B0E1114171A032069
:10AFE000C00400BD0720C00400BD0F20C00400BD88
:10AFF0001F20400300BD3F20400300BD7F204003D1
:10B0000000BDFF20400300BD084600BDFEB5264F31
:10B010000D4604000FD0002D0DD02646002020360E
:10B02000B071F07129680D208847002801DA780096
:10B03000FEBD102801D03846FEBDA562E968002992
:10B0400001D028208847204600F030F80028F3DBA4
:10B05000A06AA52182680E209047A06A9621826886
:10B060000F209047A06A0221826862209047A06A60
:10B07000002182680E209047A06A002182680F207C
:10B080009047717930200191009006232022012100
:10B090002046FFF766FE0028CEDB204600F0AEF823
:10B0A0000028C9DB0020FEBDFFFFFFFF10B586B002
:10B0B000044614216846FAF77AF8002C7ED0A06A7C
:10B0C000122143686A4610209847122877D16846B3
:10B0D000007801220101684640781203000908182F
:10B0E00043492081884201DD801A208168468378A7
:10B0F00040780007000D18186081884201DD801A31
:10B10000608168460079012201016846C078120515
:10B110000003091868464079000908183549E060BD
:10B12000884201DD801AE060684640790007030B21
:10B130006846807900021B186846C079181820619B
:10B14000884201DD801A20616846417A007A000257
:10B15000081802B2284801210904A282824201DDB6
:10B16000521AA2826A46D37A927A12029A1812B2BC
:10B17000E282824201DD521AE2826A46537B127BEE
:10B1800012029A1812B22283824201DD521A2283DD
:10B190006A46D37B927B12029A1812B26283824271
:10B1A00001DD521A62836A46537C127C12029A189D
:10B1B00012B2A283824204DD501A01E00BE008E0E3
:10B1C000A083A06A016828208847002806DA0120A9
:10B1D000C04306B010BD0020C043FAE7C011C0074D
:10B1E0002034002800D0802060710020F1E70000AA
:10B1F000FF070000FFFF0700FF7F000010B50400FD
:10B2000009D0A06A0721826808209047002805DA43
:10B210000120C04310BD0020C04310BD07202034D2
:10B220002070002010BD0000FEB5044600200190F3
:10B2300000906079734940000E5A61782578491E64
:10B240007148CFB20163042D77D0072D75D000214E
:10B250000291217801736C49E37901229205896991
:10B26000002B6CD0914381616748217A4173217A28
:10B2700082698907890B0A4382610021042000F05A
:10B2800034FB324661492E2000F024FB3846FFF79C
:10B29000F3FB5F4E0522705D810040185D49431845
:10B2A00007212B2000F030FB5B49029801220B188C
:10B2B0000B21282000F028FB705D584980000A58B7
:10B2C0000C21282000F011FBE0795549800040183E
:10B2D000A1794900425A0221272000F0FBFA514887
:10B2E0007E00825B0421272000F0F4FAE079002838
:10B2F00029D0A07804282CD0282069460872202262
:10B300000621272000F0E6FA02AB012226212720A1
:10B3100000F0FAFA444938014018E17889004258AF
:10B320000821272000F0E1FAA17A601C627A090264
:10B33000114313D016E000E001E0012188E711433A
:10B34000F608816190E764220621272000F0C2FA06
:10B35000E0E71020694608720246D1E733490172DE
:10B36000090A4172417A007A0A0202432021272009
:10B3700000F0B0FA2E4F0C2123203A6800F0B5FA05
:10B38000F01982880421232000F0A4FAA079002873
:10B390000BD0E0792749012243180021212000F039
:10B3A000B3FA03200190012000902A07120F100128
:10B3B0000243607800218007000B024301980005DA
:10B3C00002430098400402432079C006400902432A
:10B3D0006079C00602431F2000F087FAA0786178E8
:10B3E0000123084302040848DB030261E1794903B1
:10B3F00019430A4302610021082000F076FA002078
:10B40000FEBD00002CC80008BC010020042800007C
:10B41000D4C700082400002042000020DCC7000838
:10B42000FCC7000808C800080CC80008411000004C
:10B43000F4C700084400002038B50C4607498A8B41
:10B44000002102432C2000F045FA684604706B4648
:10B45000012206212C2000F057FA38BDBC01002043
:10B4600010B5FFF7F5FA10BD10B5044604213620DB
:10B4700000F0FCF80121C902002C01D0084300E0D3
:10B48000884302460421362000F02FFA10BD000048
:10B4900038B540206946087000210E2000F0E6F81B
:10B4A0000446002211460E2000F01FFA6B460122CE
:10B4B00000210D2000F028FA074A00210F2000F09B
:10B4C00014FA00F0EDF9224600210E2000F00DFAEA
:10B4D00002480021017338BDF8FF2724DC01002059
:10B4E000FEB50546042069460870514C0020607581
:10B4F00021462031206348710873A0836063A063F4
:10B5000000F0C8F84B4E206002E000F0C3F8206065
:10B51000B042FAD10020FFF7CDFA00F0BBF8464E5A
:10B5200020603078242801D9243806E00621F9F774
:10B53000DFFD0622101A40010843020601040A43F7
:10B5400001020A430243B260706000211E2000F035
:10B55000CCF900F09FF820606B46012200212420E6
:10B5600000F0D2F91E20FFF719FB86B2300AA07353
:10B570000420FFF713FB074600F08CF82060380624
:10B58000000E0DD002206946087101AB0122122184
:10B590002D2000F0B9F9A08B012109030843A083F5
:10B5A00000F078F820600620FFF7F8FA60600720C6
:10B5B000FFF7F4FAA060F006C00E207501D110204C
:10B5C0002075C0B200F0DCF9E80707D0FFF7CDFA2C
:10B5D000A08B0121C9020843A0830AE0052136207F
:10B5E00000F02EF81549084002460521362000F0EB
:10B5F00071F90120FFF75EFA0021042000F036F80F
:10B60000A0610021262000F031F8152189030843AC
:10B6100002460021262000F068F90022262136206B
:10B6200000F058F900F036F820600020FEBD000060
:10B63000BC0100203001CADE18000020FFFD000020
:10B6400038B5094C89B280B26B46022200F028F866
:10B65000002806D16846407801026846007808183C
:10B6600084B2204638BD0000FFFF000038B500243A
:10B67000E44389B280B26B46042200F011F800283E
:10B6800006D103216846435C2202D418491EFAD52C
:10B69000204638BD10B500210846FFF7E7FF10BD72
:10B6A00038B5002909D0402420436C462070C8B228
:10B6B0007F2906D8607002200AE0694608700120E0
:10B6C00006E0802420436C466070C809A070032007
:10B6D000694600F0B1FF38BD10B5144603460A466E
:10B6E00021461120FFF7DCFF10BD10B503460522EF
:10B6F00000211520FFF7D4FF10BD10B50346052229
:10B7000000211720FFF7CCFF10BD38B505460020FB
:10B710006946087000F0C4F8FF2401342246002D69
:10B7200001D00322120200210D2000F0D3F8002DD9
:10B7300013D06B46012203210F20FFF7B1FF6846AB
:10B740000078000709D5FFF7A3FE224600210D204F
:10B7500000F0C0F80020C04338BD002038BD10B54F
:10B76000024601210A2000F0C0F810BD10B50446C1
:10B7700000211A20FFF77AFF000D22030005120BAB
:10B78000024300211A2000F0B0F810BD10B50246A7
:10B7900002492E2000F09EF810BD000004180000A1
:10B7A000F8B505466B46012203210420FFF778FF18
:10B7B0000126114C3607002D0DD02A4600210C2001
:10B7C00000F088F869460878102108436946087037
:10B7D000A069304307E069460878EF2108406946D0
:10B7E0000870A069B0430B46A06101220321042028
:10B7F00000F08AF8F8BD0000BC01002010B5024638
:10B800000021182000F066F810BD0000F8B50746CA
:10B81000002568460570B807204C2E4600280ADA35
:10B820008020694608706B46012200210D2000F03F
:10B830006BF801202073F8076946087821D00621AB
:10B840000843694608706B46012200210D2000F074
:10B850005BF803210F20FFF7F3FE8121C9000842A6
:10B8600019D04020694608706B46012200210D2046
:10B8700000F04AF80020FFF7F7FD00252673ED439E
:10B8800009E002210843694608706B460122002145
:10B890000D2000F039F82846F8BD0000DC0100203A
:10B8A0001CB56B46012203210F20FFF7F9FE684605
:10B8B00000784022C1091040C9014000814208D0EF
:10B8C000012069460871024601AB03210D2000F0FA
:10B8D0001BF81CBD08B56B461A70120A5A7089B263
:10B8E00080B2022200F010F808BD38B500236C4683
:10B8F000E254120A5B1C042BFADB89B280B22346A5
:10B90000042200F001F838BD38B58024002909D0A0
:10B91000C02528436D462870C8B27F2907D86870B3
:10B92000022009E0204369460870012004E020431A
:10B930006870C809A8700320694600F027FF38BD69
:10B9400010B51446012312189B029A4202D9002016
:10B95000C04310BD0B46821E21460920FFF7D4FFCD
:10B96000002010BD10B5054A8905126901430A433C
:10B9700000210820FFF7B9FF002010BDBC01002006
:10B9800038B504466B4601220E212B20FFF788FEB6
:10B9900068460078E10640094001C90E0143684647
:10B9A00001706B4601220E212B20FFF7ADFF38BD41
:10B9B00010B5002142541C06120A22431B0A491CDE
:10B9C0000429F7DB10BD000013B501231A466946B0
:10B9D0000248FCF773FC00981CBD0000CC16002048
:10B9E0007CB5002425466846FFF77FFE04206946A3
:10B9F000220E2D02154322020C5C1443401EF7D583
:10BA0000204629467CBD7CB5002425466846FFF7C4
:10BA100074FE04206946220E2D02154322020C5C9E
:10BA20001443401EF7D5204629467CBDFBF72CF970
:10BA3000FEF7FAF8FDF708F83E493F48002522C016
:10BA400005608561C5613D490562C1600838FBF745
:10BA5000ADFAFCF7E5FFFDF7FDF8FDF799F8FCF707
:10BA6000ABFF052401222407D1032046FBF7F7F89A
:10BA7000FDF78AFEFCF788FEFAF7E8F8FAF76AF9AC
:10BA8000FAF738F9FCF79CFC0721A015FFF7D4FC66
:10BA9000FFF7E6FC012211032046FBF7E0F82648F9
:10BAA000C8222749C830FCF7D7FB264F264E274C23
:10BAB000387800280FD13078002801D003280AD127
:10BAC0000121C9022248FBF7BDF8002803D101215A
:10BAD0000846FBF77FFBE078002828D06078002834
:10BAE00025D0E57072B620780F280AD901201849B0
:10BAF00000038861FEF7E6F901201549000388621A
:10BB00000CE0012251031248FBF7A9F8FEF7DAF91D
:10BB10000121002249030E48FBF7A1F862B6FCF7A9
:10BB200059FD208C0028C3D0401E2084C0E7FCF7BC
:10BB300051FDBDE7007C004004160020FFFF00001F
:10BB4000200D00205A000020810000203C01002030
:10BB50000004005010B586B01748FBF7AAF914216D
:10BB60006846F9F724FB1548009003200190002057
:10BB70000290052069460007FAF7A8FF69461048B9
:10BB8000FAF7A4FF69460F48FAF7A0FF012108461B
:10BB9000FBF720FBFF2401342046FBF7F3FA0A49A8
:10BBA00008680422104308602046FBF7FBFAFBF705
:10BBB00001FB06B010BD000004160020FFFF0000CE
:10BBC00000040050000800500070004010B5012231
:10BBD000920217491748FAF741F9154816490288A1
:10BBE0008A4223D0018004218180FF21F531C18068
:10BBF0000A21018100211E224181D243828101223A
:10BC0000C28181834323C38602230387782343872A
:10BC10008287C28702464032118451849184C18355
:10BC2000918014238382118200F02CFD10BD00004E
:10BC3000E80D002000FC0008AA550000F0B51FB474
:10BC400096B084460C460246199D18980390490008
:10BC500068006300490840080193002A01D00126CA
:10BC600000E000269E19FE4BF6185B109E422BD377
:10BC70006E00039F0296002F00D00127F719F84E9F
:10BC8000F84BBE199E421FD3039E0346F64F334323
:10BC900009D03B469C4201D1002A04D0019B002AD6
:10BCA00005D0012604E0002039461BB0F0BD002677
:10BCB0009E19EE4B9E4207D8039F029E002F00D094
:10BCC0000127F6199E4207D92B4660462146189A4D
:10BCD000FEF788FE1BB0F0BD0023002C29DAE44EED
:10BCE000B04226DAE34EB04201DB022321E0DE4E11
:10BCF000B0421EDBE04E070DBE19142E09DD3427BD
:10BD0000BF1B039EFE400196BE40039FBE420BD068
:10BD10000FE0039F002F0CD11427BF1B0646FE40E7
:10BD20000196BE40864204D1019BDE07F60F022336
:10BD30009B1B0E46164318D1002D16DA002C03D09B
:10BD4000022B01D0012B06D00220FEF77BFEFEF76E
:10BD50003FFE1BB0F0BD0220FEF774FEFEF738FE7A
:10BD60000122D20751401BB0F0BD039E002E61D1CD
:10BD7000BF4EB04220D1C148844201D1002A08D030
:10BD8000B948814209DB002D10DB189829461BB009
:10BD9000F0BD0020B4491BB0F0BD002D06DA012231
:10BDA0002946D207189851401BB0F0BDB4497944D8
:10BDB000086849681BB0F0BDAB4FB84225D1002DD3
:10BDC0001FDA002904D0B14212D1002A09D018E0AC
:10BDD000002A72D1A649E20F0020D20711431BB0FE
:10BDE000F0BD0020E20F0146D20711431BB0F0BDA9
:10BDF000B14206DA234600203946F9F7EBFB1BB0C7
:10BE0000F0BD104621461BB0F0BDB14212DA01264A
:10BE1000B607B54203D1234610461946FEE3994EB4
:10BE2000B54207D1261E05DB1046314600F040FC26
:10BE30001BB0F0BD67007F081646002A40D10029DC
:10BE40000AD08B4A914229D1002C0EDD002D1CDB3B
:10BE5000002011461BB0F0BD022B16D0002C14D0D0
:10BE6000012B12D1002C14DB0FE0002C28DA002D5E
:10BE700009DB012B03D000207D491BB0F0BD002061
:10BE800081491BB0F0BD012B03D0002001461BB03F
:10BE9000F0BD00200121C9071BB0F0BD724A9142DC
:10BEA0000ED1002C01DA002B17D0022B06D0002077
:10BEB000C043F9F72FFC1BB0F0BD90E20120F8E77A
:10BEC000E217521C94461A4307D000220892664C8F
:10BED00062465B1E1A4307D009E00120FEF7B2FD5F
:10BEE000FEF784FD1BB0F0BD0022644C0892674A47
:10BEF00090427DDD664B674A98421FDD914202DC2D
:10BF0000002D05DB4DE05848814217DB002D48DD50
:10BF10000220FEF797FDFEF771FD05460E46002252
:10BF2000534B21460898F9F7EDFA08467100490885
:10BF3000C00FC007014328461BB0F0BD914215DA7F
:10BF4000002D2EDA0220FEF77DFDFEF757FD054697
:10BF50000E460022464B21460898F9F7D3FA7200A4
:10BF60005208C80FC0070243114617E03E4B9942E2
:10BF700023DD002D15DD0220FEF764FDFEF73EFDFA
:10BF800005460E4600223A4B21460898F9F7BAFAC0
:10BF9000084671004908C00FC007014328461BB07E
:10BFA000F0BD0220FEF74EFDFEF732FD49004908C4
:10BFB000E20FD20711431BB0F0BD002230463946D4
:10BFC000F9F792FA012205460E46D243F9F77AFBB9
:10BFD000314A324BF9F78EFA2A463346F9F792FA8C
:10BFE0000022284BF9F786FA07462A46334600E036
:10BFF00064E0039110461946F9F784FA3A46039B28
:10C00000F9F780FA0746032209915207244B284684
:10C010003146F9F777FA07910C90224A204B3846BF
:10C020000999F9F76FFA074601911F4A1F4B2846F5
:10C030003146F9F767FA3A46019BF9F755FA074690
:10C040000B460246099107990C98F9F7A9F90025C2
:10C050000E462846079B0C9AF9F746FA3A4627E01F
:10C06000FFFF1F00FFFF0F000000F03F0000E0FF98
:10C070000000F07F0000404301FCFFFF0000F0BF24
:10C08000560B00000000E03F0000F0FF0000E04120
:10C090000000F043FFFFEF3F555555555555D53F2F
:10C0A0004715F73FFE822B6544DF5DF80BAE543E2B
:10C0B000099BF9F71FFA02460B4652E101250020C1
:10C0C0002D05A94207DA352230463946F9F7FAFA42
:10C0D00006463420C0430A151218FE481018039073
:10C0E0000803FD49000B01430F46FC49884201DC6F
:10C0F000002003E0FA49884202DA0120119005E0AD
:10C10000002011900398401C7F1B03901198059705
:10C11000C200F4480F927844801843680268394698
:10C1200030460D930292F9F7DFF907910C903046F3
:10C130000D9B029A0599F9F733F902460B46002048
:10C14000E549F9F747FA09910490079B0C9AF9F72A
:10C15000D9F9129000201090E3480D467844006809
:10C160000E90012178104907084311990D9B89040D
:10C1700040180121C90447183946029A0E98F9F768
:10C18000B3F93246059BF9F7B5F902460B46294645
:10C190001098F9F7B7F9064602913B4629460E9AE0
:10C1A0001098F9F7AFF9079B0C9AF9F7A3F9324603
:10C1B000029BF9F799F9099B049AF9F7A3F90591FC
:10C1C000129A0A902B4610461946F9F79BF9064633
:10C1D0000246C6480F460B4606217844FEF7A2FBEE
:10C1E00032463B460091049010461946F9F78AF909
:10C1F000009B049AF9F786F906460F462B46194626
:10C20000129A1098F9F7CCF8059B0A9AF9F77AF97F
:10C2100032463B46F9F7C4F8109A079104902B4632
:10C2200010461946F9F76EF9B14E002233460991CE
:10C230000290F9F7B5F8079B049AF9F7B1F80020D6
:10C240000746024633460091F9F74EF9099B029AD8
:10C25000F9F74AF9079B049AF9F74CF906460D914C
:10C260003A462946009B1098F9F74CF907910C9033
:10C270002B463046129A0D99F9F744F905460E46B9
:10C280003A46009B05990A98F9F73CF933462A4645
:10C29000F9F786F802460B460746099107990C986C
:10C2A000F9F77EF800250E462846079B0C9AF9F709
:10C2B0001BF93A46099BF9F71DF907460722099130
:10C2C00052078C4B31462846F9F71CF9079100902C
:10C2D000894A884B38460999F9F714F907460191BC
:10C2E000864A874B31462846F9F70CF93A46019BB6
:10C2F000F9F756F8834B7B440F9A9B181A685B68D2
:10C30000F9F74EF8029009910398F9F703FA0591AD
:10C310000490099B029A07990098F9F741F87A4B23
:10C320007B440F9A9B181A685B6817460393F9F7CA
:10C3300037F8059B049AF9F733F80E462846059B13
:10C34000049AF9F7D1F83A46039BF9F7CDF8079B21
:10C35000009AF9F7C9F8099B029AF9F7CBF8024657
:10C360000B46199900200C900F461898F9F7CAF857
:10C37000029104903B460C9A19991898F9F7B4F871
:10C380002A463346F9F7BEF8029B049AF9F708F8F3
:10C3900009910E902A46334639460C98F9F7B2F8BF
:10C3A00006460F46099B0E9AF8F7FAFF574A0D46C4
:10C3B000914220DB5242AA18024310D132463B463A
:10C3C000F9F792F804900391514A524B09990E984B
:10C3D000F8F7E6FF039B049AF9F756FA1ED20220FB
:10C3E000FEF730FBFEF70AFB49004908E20FD207CF
:10C3F00011431BB0F0BD6A00474B52089A420DD35F
:10C40000464AAA18024300D0CBE532463B46F9F72C
:10C410006BF8099B0E9AF9F737FAF5D968000023F3
:10C4200040082C490393020D3D4B5218984223DDDE
:10C4300001200005521CD04042195000400D401808
:10C4400038497944096813468C463749C1408B43C3
:10C4500012030121120B090551181422101AC140B0
:10C460000391002D01DA4842039062463046394676
:10C47000F9F73AF806460F4632463B4609990E98B8
:10C48000F8F78EFF00252A46284B28460591F9F734
:10C4900039F807910C90264A264B28460599F9F75A
:10C4A00031F80091029032463B4628460599F9F74B
:10C4B0001BF8099B0E9AF9F71DF81F4A1F4BF9F755
:10C4C00021F8009B029AF8F76BFF07460B460246DD
:10C4D000099135E001FCFFFF0000F03F8E9803005A
:10C4E0007AB60B0066070000A8070000D20600001D
:10C4F0000000084009C7EE3FFD033ADCF5015B147C
:10C50000E02F3EBEA60500006C0500000000904034
:10C51000FE822B654715973C00CC904000346F3F5E
:10C520000000E03FC2040000FFFF0F00432EE63F83
:10C53000396CA80C615C20BEEF39FAFE422EE63F52
:10C5400007990C98F8F72CFF05460E46079B0C9AA6
:10C55000F8F7CAFF3A46099BF8F7CCFF09912A463B
:10C5600033460E9010461946F8F7CCFF07460246B0
:10C570002F480B46059105217844FEF7D3F93A463A
:10C58000059BF8F7BFFF2A463346F8F7B3FF074687
:10C59000019128463146099B0E9AF8F7B3FF099B93
:10C5A0000E9AF8F7FDFE012304910C9000229B07E0
:10C5B00038460199F8F798FF05910E903A462846BB
:10C5C0003146019BF8F79EFF059B0E9AF9F702F89A
:10C5D000049B0C9AF8F788FF2A463346F8F784FF45
:10C5E0000022144BF8F786FF064603980D46000517
:10C5F00041190915002912DC30462946039AF9F73A
:10C6000061F8FEF749F9042801D1FEF701FA304636
:10C610002946039AF9F756F8064601E004E029187E
:10C620000B46324621460898F8F76CFF1BB0F0BD68
:10C63000640300000000F03FF0B58C460025102692
:10C64000052109078E620E4C08E067467F5DE760B2
:10C65000A768FF07FCD0E7681F706D1C8542F4DBFC
:10C660000020074606E0E760A568ED07FCD0E56816
:10C670001D54401C9042F6D38E610020F0BD000096
:10C680000030014070B572B60124074DA402214666
:10C690002846F9F7C9FB002804D02246034928465A
:10C6A000F9F766FC62B670BD00FC0008E80D0020DA
:10C6B000F8B506460C46F9F7F5F9051E0F4600D009
:10C6C0000120014349000B484908411AC90F0DD008
:10C6D000002E01D0012100E000210C436100490837
:10C6E000401AC00F02D10120FEF7ACF928463946A6
:10C6F000F8BD00000000F07FF8B515460E4607466D
:10C70000002407E03819C0B200F008F8641C287053
:10C71000E4B26D1CB442F5D33046F8BD10B5044602
:10C72000FBF7F4FEEE20FBF7C4FEFBF728FF2046E4
:10C73000FBF7BFFEFBF723FFFBF7E8FEEF20FBF75D
:10C74000B8FEFBF71CFF0020FBF786FE0446FBF754
:10C75000F8FE204610BD704770B50D460446FBF745
:10C76000D5FEEE20FBF7A5FEFBF709FF2046FBF701
:10C77000A0FEFBF704FF2846FBF79BFEFBF7FFFE3E
:10C78000FBF7DFFE0A20FEF7A6FA70BDF0B5002524
:10C79000102605279C463F070B46BE620C4C06E060
:10C7A000595DE160A168C907FCD0E1686D1C854254
:10C7B000F6DB002007E06146095CE160A168C9077B
:10C7C000FCD0E168401C9042F5D3BE610020F0BD72
:10C7D000003001400000010203040005405C00003D
:10C7E000A05C0400C06C0800805C0400E03F1E00F8
:10C7F000E07D1E0007A9022570889B880A001600AC
:10C80000010006000100020087008D002D001A3192
:10C8100052001A339A001A351D011A376B003B314A
:10C82000BE003B335E013B3596023B370000995911
:10C830009959EB518F421E45142E0080EB51F5287B
:10C840003333E13A703DE13AC235852BC23533339B
:10C85000C235C235AE47E13A5138A33051380000F5
:10C860000000000000000102030406070809030499
:10C8700006080C101820300000000001020304001C
:10C88000000000000000F03F000000000000F83F42
:10C8900000000000000000000000004003B8E23F7C
:10C8A000000000000000000006D0CF43EBFD4C3E2E
:10C8B000033333333333E33FFFAB6FDBB66DDB3F23
:10C8C0004D268F515555D53F01411DA96074D13F6B
:10C8D00065DBC9934A86CD3FEF4E454A287ECA3F65
:10C8E0003E5555555555C53F93BDBE166CC166BFE7
:10C8F0002CDE25AF6A56113FF16BD2C541BDBBBEE0
:10C90000D0A4BE726937663E00000000000000003F
:10C9100030C9000800000020900100006C5B000896
:10C9200094C9000890010020681A000034AA000889
:10C930000124130704380D091E08054008260910B4
:10C940004008560A131D043B08BE0516D8BC40100B
:10C950000852010338C842077252030CE5800C1BD1
:10C960000202DD140901022281F01F668104988908
:10C970009686967982159803981498879674977876
:10C9800082439788967197778249F10139293F92BE
:04C9900004922000ED
:04000005080050C1DE
:00000001FF
